:020000040000FA
:10000000F0EF37F0C96E1200CEEF33F057EC10F07E
:10001000E1EC14F0FDD7120043EF36F0D9CFE5FF45
:10002000E1CFD9FF00C0E5FF01C0E5FF02C0E5FF59
:1000300003C0E5FF04C0E5FF05C0E5FF06C0E5FF1E
:1000400007C0E5FF08C0E5FF09C0E5FF0AC0E5FFFE
:100050000BC0E5FF0CC0E5FF0DC0E5FF0EC0E5FFDE
:100060000FC0E5FF10C0E5FF11C0E5FF12C0E5FFBE
:1000700013C0E5FF14C0E5FF15C0E5FF16C0E5FF9E
:1000800017C0E5FF18C0E5FF19C0E5FF1AC0E5FF7E
:100090001BC0E5FF1CC0E5FF1DC0E5FF1EC0E5FF5E
:1000A0001FC0E5FF20C0E5FF21C0E5FF22C0E5FF3E
:1000B00023C0E5FF24C0E5FF25C0E5FF020EDBCF2E
:1000C00000F0030EDBCF01F0040EDBCF02F0025094
:1000D000086E0150076E0050066EE56A100EE56E60
:1000E0000850E56E0750E56E0650E56E800EE56E31
:1000F000040EE56EE80EE56EB4EC2AF0080EE1267B
:10010000F0C403F0F1C404F0F2C405F0F3C406F047
:1001100003C007F004C008F005C009F006C00AF0EB
:10012000D8800AAED8900AE30A1E091E081E076C82
:1001300005E1082A03E1092AD8B40A2AE8C40BF029
:10014000E9C40CF0E86A0401E9BFFF0E0D6E0E6E03
:10015000D890EC31106EEB310F6ED89010320F3218
:10016000ED51E840E840C00B1012ED41E8403F0B74
:10017000E8BAC009116E126A11BE12680F500B5C0A
:100180000F6E10500C58106E11500D58116E125009
:100190000E58126E800F810F08E1FF0E115C05E111
:1001A000FF0E105C02E1FE0E0F5CD8A04ED0125084
:1001B000800F800F08E1000E115C05E1000E105C5D
:1001C00002E1030E0F5CD8B040D00A340A30166E3C
:1001D0000930156E0830146E0730136EF6C417F030
:1001E000F7C418F0E86A0401F7BFFF0E196E800F1C
:1001F000F36E1650800FF35C08E11550195C05E1B1
:100200001450185C02E11350175C1FE30C50156E7C
:1002100015260D34166ED890153616360B44E84464
:10022000FC0B146E0B50E844E844030B1512040158
:10023000EA6B1450EB6F1550EC6F1650ED6FF06BCE
:10024000F16BF26BF36BB0EF04F00850076E0950DE
:10025000086ED89008320732D890083207320A5018
:10026000E840E840C00B08120A40E8403F0BE8BAFB
:10027000C0090A6A083408300A6E0730096EE86A55
:100280000ABEFF0E0B6E0C6E07C00DF008C00EF01C
:10029000E86A08BEFF0E136EE56E1350E56E0E5051
:1002A000E56E0D50E56E0C50E56E0B50E56E0A5094
:1002B000E56E0950E56E91EC22F0096EF3CF0AF07D
:1002C000F4CF0BF0E9CF0CF0080EE126F6C40DF0E8
:1002D000F7C40EF0E86A0401F7BFFF0E136E146E48
:1002E000E56E1350E56E0E50E56E0D50E56E0C5048
:1002F000E56E0B50E56E0A50E56E0950E56E79EC3F
:1003000025F0096EF3CF0AF0080EE126EEC40BF0DB
:10031000EFC40CF0E86A0401EFBFFF0E156E0C503D
:10032000196E192615341A6ED89019361A360B44E0
:10033000E844FC0B186E0B50E844E844030B191218
:10034000176AD88006AED890D8B064D109C00BF037
:100350000AC00CF0E86A0ABEFF0E156E800FF36E3D
:100360001250800FF35C08E11150155C05E110504C
:100370000C5C02E10F500B5CD8B024D10650800F0A
:10038000F36E1A50800FF35C08E11950055C05E12B
:100390001850045C02E11750035CD8B0ECD0F4C4F0
:1003A0000BF0F5C40CF0E86A0401F5BFFF0E156E02
:1003B000166E03500B2604500C22055015220650D1
:1003C00016220B500401F06F0C50F16F1550F26FB4
:1003D0001650F36FF6C40BF0F7C40CF0F4C415F02C
:1003E000F5C416F00C50800FF36E1650800FF35CBE
:1003F00002E115500B5CD8B0A2D0F0C41BF0F1C4E0
:100400001CF0F2C41DF0F3C41EF0D8901D30206E15
:100410001C301F6ED89020321F321E50E840E8403A
:10042000C00B20121E40E8403F0BE8BAC009226A08
:100430001F50076E2050086E08340830206E0730B9
:100440001F6EE86A20BEFF0E216E226E07C023F0E9
:1004500008C024F0E86A08BEFF0E256EE56E255040
:10046000E56E2450E56E2350E56E2250E56E215076
:10047000E56E2050E56E1F50E56E91EC22F01F6E88
:10048000F3CF20F0F4CF21F0E9CF22F0080EE126DF
:100490000BC023F00CC024F0E86A0CBEFF0E256EE2
:1004A000E56E2550E56E2450E56E2350E56E225032
:1004B000E56E2150E56E2050E56E1F50E56E79EC3B
:1004C00025F01F6EF3CF20F0080EE1261F50096EB5
:1004D00020500A6E09C01FF00AC020F0E86A0ABE68
:1004E000FF0E216E226E1250800FF36E2250800F8D
:1004F000F35C08E12150115C05E12050105C02E141
:100500001F500F5C1CE20B50155C0B6E0C50165804
:100510000C6EE86A0CBEFF0E156E166E0B501B5E5D
:100520000C501C5A15501D5A16501E5A1B500401CF
:10053000F06F1C50F16F1D50F26F1E50F36F1A5088
:10054000800FF36E0401F351800FF35C08E1F25168
:10055000195C05E1F151185C02E1F051175CD8B06B
:10056000D8D117500401F06F1850F16F1950F26F85
:100570001A50F36FCED11A50800FF36E0650800FD1
:10058000F35C08E10550195C05E10450185C02E1D8
:100590000350175CD8B0BDD10D50035C0B6E0E50EC
:1005A00004580C6E13500558156E14500658166EEC
:1005B0000B500401F06F0C50F16F1550F26F165094
:1005C000F36FA7D1F4C40BF0F5C40CF0E86A040192
:1005D000F5BFFF0E156E166E0D500B260E500C2239
:1005E00013501522145016220B50035C0B6E0C5046
:1005F00004580C6E15500558156E16500658166E98
:100600000B500401F06F0C50F16F1550F26F165043
:10061000F36F7FD10A1E096CD8B40A2A09C00BF007
:100620000AC00CF0E86A0ABEFF0E156E166E125074
:10063000800FF36E1650800FF35C08E11550115CCB
:1006400005E10C50105C02E10B500F5CD8B03ED1BC
:100650001A1C166E191C156E181C0C6E171C0B6ECE
:100660000B2A04E10C2A02E1154A162A1650800FC3
:10067000F36E0650800FF35C08E10550155C05E150
:1006800004500C5C02E103500B5CD8B0F8D0F4C409
:1006900017F0F5C418F0E86A0401F5BFFF0E196EF3
:1006A0001A6E1750035C176E18500458186E1950C4
:1006B0000558196E1A5006581A6E17500401F06F3B
:1006C0001850F16F1950F26F1A50F36FF6C417F00B
:1006D000F7C418F0F4C419F0F5C41AF01850800FDC
:1006E000F36E1A50800FF35C02E11950175CD8B01A
:1006F000AAD0F0C41BF0F1C41CF0F2C41DF0F3C486
:100700001EF0D8901D30206E1C301F6ED890203205
:100710001F321E50E840E840C00B20121E40E84047
:100720003F0BE8BAC009216E226A21BE2268221E50
:10073000211E201E1F6C05E1202A03E1212AD8B4C6
:10074000222A1F50076E2050086E08340830206E91
:1007500007301F6EE86A20BEFF0E216E226EE86A27
:1007600008BEFF0E236EE56E2350E56E0850E56E61
:100770000750E56E2250E56E2150E56E2050E56E83
:100780001F50E56E91EC22F0076EF3CF08F0F4CF26
:100790001FF0E9CF20F0080EE12617C021F018C0A5
:1007A00022F0E86A18BEFF0E236EE56E2350E56E58
:1007B0002250E56E2150E56E2050E56E1F50E56E2B
:1007C0000850E56E0750E56E79EC25F0076EF3CF23
:1007D00008F0080EE126081E076C02E1082A00E175
:1007E0000750096E08500A6EE86A0ABEFF0E076ECF
:1007F000800FF36E1250800FF35C08E11150075C1C
:1008000005E110500A5C02E10F50095C1CE2175030
:10081000195C176E18501A58186EE86A18BEFF0E49
:10082000076E086E17501B2618501C2207501D22F9
:1008300008501E221B500401F06F1C50F16F1D5018
:10084000F26F1E50F36F0401F351800FF36E1650D8
:10085000800FF35C08E11550F25D05E10C50F15D8D
:1008600002E10B50F05DD8B054D00B500401F06F92
:100870000C50F16F1550F26F1650F36F4AD00650BE
:10088000800FF36E1650800FF35C08E11550055C85
:1008900005E10C50045C02E10B50035CD8B039D088
:1008A0000D500324076E0E500420086E13500520CF
:1008B000096E145006200A6E07500401F06F0850AC
:1008C000F16F0950F26F0A50F36F23D0F4C407F0B0
:1008D000F5C408F0E86A0401F5BFFF0E096E0A6E60
:1008E00007500D2608500E22095013220A501422D8
:1008F0000D5003260E5004221350052214500622D8
:1009000003500401F06F0450F16F0550F26F065070
:10091000F36FD8900401F231046EF131036ED89078
:1009200004320332F351E840E840C00B0412F341B3
:10093000E8403F0BE8BAC009056E066A05BE0668C6
:10094000EA510326EB510422EC510522ED51062217
:100950000350EA6F0450EB6F0550EC6F0650ED6FDB
:10096000E56A100EE56E800EE56E040EE56EE80E8B
:10097000E56E0250E56E0150E56E0050E56EB4EC98
:100980002AF0080EE126E4CF25F0E4CF24F0E4CFEE
:1009900023F0E4CF22F0E4CF21F0E4CF20F0E4CF45
:1009A0001FF0E4CF1EF0E4CF1DF0E4CF1CF0E4CF45
:1009B0001BF0E4CF1AF0E4CF19F0E4CF18F0E4CF45
:1009C00017F0E4CF16F0E4CF15F0E4CF14F0E4CF45
:1009D00013F0E4CF12F0E4CF11F0E4CF10F0E4CF45
:1009E0000FF0E4CF0EF0E4CF0DF0E4CF0CF0E4CF45
:1009F0000BF0E4CF0AF0E4CF09F0E4CF08F0E4CF45
:100A000007F0E4CF06F0E4CF05F0E4CF04F0E4CF44
:100A100003F0E4CF02F0E4CF01F0E4CF00F0E4CF44
:100A2000D9FF1200D9CFE5FFE1CFD9FF00C0E5FF24
:100A300001C0E5FF02C0E5FF03C0E5FF04C0E5FF1C
:100A400005C0E5FF06C0E5FF07C0E5FF08C0E5FFFC
:100A500009C0E5FF0AC0E5FF0BC0E5FF0CC0E5FFDC
:100A60000DC0E5FF0EC0E5FF0FC0E5FF10C0E5FFBC
:100A700011C0E5FF12C0E5FF13C0E5FF14C0E5FF9C
:100A800015C0E5FF16C0E5FF17C0E5FF18C0E5FF7C
:100A900019C0E5FF1AC0E5FF1BC0E5FF1CC0E5FF5C
:100AA0001DC0E5FF1EC0E5FF020EDBCF00F0030E08
:100AB000DBCF01F0040EDBCF02F0050EDBCF03F03D
:100AC000060EDBCF04F0070EDBCF05F0080EDBCF00
:100AD00006F0090EDBCF07F00A0EDBCF08F0096A3B
:100AE0000A6A02C00DF00D50800A0DE102500101AA
:100AF0005F6F01505E6F00505D6F010E016E5D0E05
:100B0000006E800E026E03C0E9FF04C0F3FF0550C3
:100B100029EC38F00B6E0B50D8B400EF09F00B50F5
:100B2000250A02E0E7EF08F00C6A0D6A0E6A0F6A08
:100B3000106A0A0E116E126A136A146A200E156E7C
:100B40001668176A2B0E186E032A02E3044A052A58
:100B500003C0E9FF04C0F3FF055029EC38F0196E1B
:100B6000250A13E11950E56E0250E56E0150E56E5D
:100B70000050E56E2BEC2AF0040EE126094A0A2A01
:100B8000032A02E3044A052ABED71950300A06E1B7
:100B9000300E156E032A02E3044A052A03C0E9FF5A
:100BA00004C0F3FF055029EC38F02D0A06E1010ED0
:100BB000146E032A02E3044A052A03C0E9FF04C0B5
:100BC000F3FF055029EC38F0200A08E1010E176EFA
:100BD000200E186E032A02E3044A052A03C0E9FF27
:100BE00004C0F3FF055029EC38F02B0A06E1010E92
:100BF000176E032A02E3044A052A03C0E9FF04C072
:100C0000F3FF055029EC38F0196E800F4F0F2DE3DC
:100C10001950800F460F29E203C019F004C01AF0E2
:100C200005C01BF019C0E9FF1AC0F3FF1B5029ECE7
:100C300038F01C6E800F500F12E31C50800F460FCF
:100C40000EE213500A0DF3CF1DF01D501C26D00EDE
:100C50001C24136E192A02E31A4A1B2AE3D719C06F
:100C600003F01AC004F01BC005F003C0E9FF04C084
:100C7000F3FF055029EC38F02E0A2EE1032A02E397
:100C8000044A052A166A03C019F004C01AF005C008
:100C90001BF019C0E9FF1AC0F3FF1B5029EC38F014
:100CA0001C6E800F500F12E31C50800F460F0EE297
:100CB00016500A0DF3CF1DF01D501C26D00E1C241B
:100CC000166E192A02E31A4A1B2AE3D719C003F049
:100CD0001AC004F01BC005F003C0E9FF04C0F3FF15
:100CE000055029EC38F0196E6C0A07E1010E0C6E04
:100CF000032A02E3044A052A09D01950680A06E1CA
:100D0000010E0E6E032A02E3044A052A03C0E9FF1E
:100D100004C0F3FF055029EC38F0750A06E1010E16
:100D2000106E032A02E3044A052A03C0E9FF04C047
:100D3000F3FF055029EC38F0196E730A05E1010E36
:100D40000D6E200E156E3FD01950780A03E1100E7B
:100D5000116E39D01950580A05E1100E116E010EAE
:100D6000126E31D01950630A02E1116A2CD0195069
:100D70006F0A03E1080E116E26D01950660A03E1CE
:100D8000010E0F6E20D01950640A1DE01950690A37
:100D90001AE0105005E0FF0E03260422052213D0AE
:100DA0001950E56E0250E56E0150E56E0050E56E9B
:100DB0002BEC2AF0040EE126094A0A2A032A02E350
:100DC000044A052AA0D60D5021E00650030F0D6EEF
:100DD000000E0720196E000E08201A6E0DC006F0D6
:100DE00019C007F01AC008F0FD0E0D26FF0E1922DB
:100DF0001A220DC0E9FF19C0F3FF1A5005EC37F0B5
:100E00000D6EF3CF19F0F4CF1AF032D10F50D8B4E1
:100E10003ED00650040F0F6E000E07201B6E000E12
:100E200008201C6E0FC006F01BC007F01CC008F0A5
:100E3000FC0E0F26FF0E1B221C220FC0E9FF1BC059
:100E4000F3FF1C508BEC36F00F6EF3CF1BF0F4CF9A
:100E50001CF0E9CF1DF0040E196E000E0D6E800E11
:100E60001A6E1650E56E240EE56E040EE56E000E49
:100E7000E56E1D50E56E1C50E56E1B50E56E0F5083
:100E8000E56E7FEC21F0080EE1261668F1D01668B9
:100E90000C5023E00650040F0C6E000E07200F6E5E
:100EA000000E08201B6E0CC006F00FC007F01BC020
:100EB00008F0FC0E0C26FF0E0F221B220CC0E9FFCF
:100EC0000FC0F3FF1B508BEC36F00C6EF3CF0FF01E
:100ED000F4CF1BF0E9CF1CF06AD00E5032E0065080
:100EE000020F0E6E000E07201D6E000E08201E6EF3
:100EF0000EC006F01DC007F01EC008F0FE0E0E2644
:100F0000FF0E1D221E220EC0E9FF1DC0F3FF1E5062
:100F1000C4EC37F00E6E0EC00CF0E86A0EBEFF0E89
:100F20000F6E1B6E1C6E11500A0A03E11050D8B4EC
:100F30003ED00C500E6E0EC00CF00F6A1B6A1C6A7D
:100F400036D00650020F0E6E000E07201D6E000EEA
:100F500008201E6E0EC006F01DC007F01EC008F06F
:100F6000FE0E0E26FF0E1D221E220EC0E9FF1DC022
:100F7000F3FF1E50C4EC37F00E6EF3CF1DF00EC021
:100F80000CF01DC00FF0E86A1DBEFF0E1B6E1C6E3C
:100F900011500A0A02E110500AE00C500E6E0F5078
:100FA0001D6E0EC00CF01DC00FF01B6A1C6A040EF3
:100FB000196E010E0D6E800E1A6E1150D8B440D00D
:100FC000105013E01150E56E040EE56E010EE56E53
:100FD0001C50E56E1B50E56E0F50E56E0C50E56E33
:100FE0009DEC24F0070EE12612D01150E56E040EA0
:100FF000E56E010EE56E1C50E56E1B50E56E0F5060
:10100000E56E0C50E56E49EC2EF0070EE126175008
:101010002FE00DC0E9FF19C0F3FF1A5029EC38F09A
:101020002D0A26E0FF0E0D2619221A2218C0E5FF10
:101030000DC0E9FF19C0F3FF1A50B7EC38F018D013
:101040000CC0E5FF0DC0E9FF19C0F3FF1A50B7EC63
:1010500038F00D50010F0C6E000E19200E6E000EB0
:101060001A20E56A0CC0E9FF0EC0F3FFB7EC38F0B8
:101070000DC00CF019C00EF01AC00FF013C010F024
:10108000105010E00CC0E9FF0EC0F3FF0F5029EC28
:1010900038F0176E175006E00C2A02E30E4A0F2AAA
:1010A0001006EED710C013F014501EE109C00CF06A
:1010B0000AC00EF010C00FF00F5010E01550E56E92
:1010C0000250E56E0150E56E0050E56E2BEC2AF003
:1010D000040EE1260C4A0E2A0F06EED70CC009F0CA
:1010E0000EC00AF00FC013F016C00CF00DC00DF0CA
:1010F00019C00EF01AC00FF009C010F00AC015F0A8
:101100000DC0E9FF0EC0F3FF0F5029EC38F0166E4A
:101110001650D8B43ED00CC016F0176A161E171E13
:101120001650171005E00CC016F00C06165031E0F2
:101130000DC0E9FF0EC0F3FF0F5029EC38F0116E1F
:10114000125010E01150E56E81EC37F0166EE65249
:10115000165004E01150166E169A02D011C016F007
:1011600016C011F01150E56E0250E56E0150E56EAB
:101170000050E56E2BEC2AF0040EE1260D2A02E366
:101180000E4A0F2A104A152A1350D8B4B9D713069D
:10119000B7D710C009F015C00AF014502BE010C0EA
:1011A0000CF015C00DF013C00EF00E501FE0200E15
:1011B000E56E0250E56E0150E56E0050E56E2BECD9
:1011C0002AF0040EE1260C4A0D2A0E06EED70B502B
:1011D000E56E0250E56E0150E56E0050E56E2BECB9
:1011E0002AF0040EE126094A0A2A04D00CC009F0AC
:1011F0000DC00AF0032A02E3044A052A83EF05F032
:101200000AC0F3FF0950E4CF1EF0E4CF1DF0E4CF95
:101210001CF0E4CF1BF0E4CF1AF0E4CF19F0E4CFD8
:1012200018F0E4CF17F0E4CF16F0E4CF15F0E4CFD8
:1012300014F0E4CF13F0E4CF12F0E4CF11F0E4CFD8
:1012400010F0E4CF0FF0E4CF0EF0E4CF0DF0E4CFD8
:101250000CF0E4CF0BF0E4CF0AF0E4CF09F0E4CFD8
:1012600008F0E4CF07F0E4CF06F0E4CF05F0E4CFD8
:1012700004F0E4CF03F0E4CF02F0E4CF01F0E4CFD8
:1012800000F0E4CFD9FF1200D9CFE5FFE1CFD9FFBD
:1012900000C0E5FF01C0E5FF02C0E5FF03C0E5FFB8
:1012A00004C0E5FF05C0E5FF06C0E5FF07C0E5FF98
:1012B00008C0E5FF09C0E5FF0AC0E5FF0BC0E5FF78
:1012C0000CC0E5FF0DC0E5FF020EDBCF00F0030E02
:1012D000DBCF01F0040EDBCF02F00050090F066EE9
:1012E000000E0120076E000E0220086E0B6E0750E4
:1012F0000A6E0650096EE56A0D0EE56E0B50E56E3E
:101300000A50E56E0950E56E800EE56E010EE56E41
:101310001F0EE56EB4EC2AF0080EE12600C009F0BD
:1013200001C00AF002C00BF0E56AE56E0B50E56EF5
:101330000A50E56E0950E56E800EE56E040EE56E0E
:10134000810EE56EB4EC2AF0080EE12681C403F0AC
:101350000350010A04E00350030A01E01FD1010118
:1013600027510101345D036E0101285101013559F6
:10137000046E010129510101365901012A5101016F
:10138000375903500101666F0450676F01013451F2
:101390000101276F010135510101286F010136510B
:1013A0000101296F0101375101012A6F01016651C5
:1013B0006711D8A47FD02DEC35F0036EF3CF04F085
:1013C000F4CF05F0E9CF09F001012C510A6E2D513F
:1013D0000B6E2E510C6E2F510D6E0A50035E0B508A
:1013E000045A0C50055A0D50095A03500401FC6F61
:1013F0000450FD6F0550FE6F7F0E0914FF6F010151
:101400002BB125D00401FD35FF31046EFE31036E92
:10141000043404320332000E04BEFF0E096E056E62
:1014200086C40AF00B6A0C6A0D6A0D50800FF36EC9
:101430000950800FF35C08E105500C5C05E1045095
:101440000B5C02E103500A5C02E201012B81010105
:101450002BB14AD023C103F024C104F025C105F00B
:1014600026C109F00401FF51800FF36E0950800F6F
:10147000F35C08E10550FE5D05E10450FD5D02E10D
:101480000350FC5D08E203C0FCF404C0FDF405C099
:10149000FEF409C0FFF4010138A303D0010E036E6E
:1014A00001D0036803C066F10101676B03AE01D090
:1014B00067691AD001012B9130C1FCF431C1FDF4F0
:1014C00032C1FEF433C1FFF40401FC510101236F6A
:1014D0000401FD510101246F0401FE510101256F3A
:1014E0000401FF510101266F0401FF51800F800F9D
:1014F00008E1000EFE5D05E1000EFD5D02E1010E5A
:10150000FC5D06E20A01F56BF66BF76BF86B46D0F3
:101510000401FC51036EFD51046EFE51056EFF5136
:10152000E56E0550E56E0450E56E0350E56E010E64
:10153000E56E000EE56AE56AE56A16EC29F0036ED1
:10154000F3CF04F0F4CF05F0E9CF09F0080EE1265F
:1015500066C10AF067C10BF0E86A010167BFFF0EC0
:101560000C6E0D6E0950E56E0550E56E0450E56E8B
:101570000350E56E0D50E56E0C50E56E0B50E56EB8
:101580000A50E56E91EC22F00A01F56FF3CFF6FAFE
:10159000F4CFF7FAE9CFF8FA080EE126020E0401BB
:1015A000815DD8A045D1010138A142D10050230F5F
:1015B000036E000E0120046E000E0220E56E045042
:1015C000E56E0350E56E0EEC00F0030EE1260050D0
:1015D000230F036E000E0120046E000E0220056E24
:1015E000020E0326000E0422052203C0E9FF04C0F8
:1015F000F3FF05508BEC36F0F3CF04F0F4CF05F099
:10160000E9CF09F00450036E0550046ED8900432FF
:101610000332D890043203320950E840E840C00B4E
:1016200004120940E8403F0BE8BAC009056E096A98
:1016300005BE096801013451035C0A01F96F01011B
:10164000355104580A01FA6F0101365105580A0153
:10165000FB6F0101375109580A01FC6FD880FCAFBC
:10166000D89022E30401831D046E821D036E034A99
:10167000042AE86A04BEFF0E056E096E0A01FC51D9
:10168000800FF36E0950800FF35C08E10550FB5D9D
:1016900005E10450FA5D02E10350F95D05E30A013A
:1016A000F96BFA6BFB6BFC6B0A01FC51800F800F2E
:1016B00008E1000EFB5D05E1000EFA5D02E1010E9E
:1016C000F95D1EE382C403F083C404F0E86A0401F8
:1016D00083BFFF0E056E800FF36E0A01FC51800F71
:1016E000F35C08E1FB51055C05E1FA51045C02E1A1
:1016F000F951035C05E30A01F96BFA6BFB6BFC6BB8
:101700000401875109E0E86CD8900A01F937FA37EB
:10171000FB37FC37010FF9E30A01FC51800F800F02
:1017200008E1000EFB5D05E1800EFA5D02E1000EAE
:10173000F95D07E30A01F9697F0EFA6FFB6BFC6B39
:1017400014D00A01FC51800F810F08E1FF0EFB5DF0
:1017500005E1800EFA5D02E1000EF95D06E20A0184
:10176000F96B800EFA6FFB69FC690050330F036E52
:10177000000E0120046E000E0220056E0A01F951D0
:10178000096EFA51E56E0950E56E0550E56E04509C
:10179000E56E0350E56E16EC17F0050EE126040128
:1017A0008151030A23E10050330F036E000E012024
:1017B000046E000E0220056E0B0E0326000E04229E
:1017C000052203C0E9FF04C0F3FF05508BEC36F09F
:1017D000F3CF04F0F4CF05F00450036E0550046E0F
:1017E000035001011F6F0450206F22D00050330FAF
:1017F000036E000E0120046E000E0220056E0B0E1B
:101800000326000E0422052203C0E9FF04C0F3FFF3
:1018100005508BEC36F0F3CF04F0F4CF05F0045014
:10182000036E0550046E03500101216F0450226FB6
:1018300081C403F00350010A04E00350030A01E0ED
:101840007DD01FC103F020C104F0E86A010120BF70
:10185000FF0E056E096E0A01F551035C0A01F96F6E
:101860000A01F65104580A01FA6F0A01F7510558A6
:101870000A01FB6F0A01F85109580A01FC6F800F39
:10188000800F08E1000EFB5D05E1800EFA5D02E1CC
:10189000000EF95D07E30A01F9697F0EFA6FFB6B31
:1018A000FC6B14D00A01FC51800F810F08E1FF0E80
:1018B000FB5D05E1800EFA5D02E1000EF95D06E2D6
:1018C0000A01F96B800EFA6FFB69FC690050440F46
:1018D000036E000E0120046E000E0220056E0A0148
:1018E000F951096EFA51E56E0950E56E0550E56E45
:1018F0000450E56E0350E56E16EC17F0050EE12678
:10190000440E0026000E012202220B0E0026000EBD
:101910000122022200C0E9FF01C0F3FF02508BEC5C
:1019200036F0F3CF01F0F4CF02F00150006E025018
:10193000016E00500101216F0150226F0850086EA6
:10194000E56A0D0EE56E800EE56E010EE56E1F0E6A
:10195000E56E0850E56E0750E56E0650E56EB4EC96
:101960002AF0080EE126E4CF0DF0E4CF0CF0E4CF2E
:101970000BF0E4CF0AF0E4CF09F0E4CF08F0E4CFB5
:1019800007F0E4CF06F0E4CF05F0E4CF04F0E4CFB5
:1019900003F0E4CF02F0E4CF01F0E4CF00F0E4CFB5
:1019A000D9FF120025642025640A000005C0E5FF68
:1019B00006C0E5FF07C0E5FF08C0E5FF09C0E5FF79
:1019C0000AC0E5FF0BC0E5FF0CC0E5FF0DC0E5FF59
:1019D0000EC0E5FF0FC0E5FF10C0E5FF11C0E5FF39
:1019E00012C0E5FF13C0E5FF14C0E5FF15C0E5FF19
:1019F00016C0E5FF17C0E5FF18C0E5FF19C0E5FFF9
:101A00001AC0E5FF1BC0E5FF1CC0E5FF1DC0E5FFD8
:101A1000000E00B0050F066AF60F02E3062AFCD797
:101A20000A0F056E042E03D0FB0F01E3062A0650B1
:101A300000B0020F00B2050F076AF60F02E3072A93
:101A4000FCD70A0F066E042E03D0FB0F01E3072A12
:101A5000075000B0060F00B2020F00B4050F086A6D
:101A6000F60F02E3082AFCD70A0F076E042E03D0F4
:101A7000FB0F01E3082A085000B2010F00B4020F67
:101A800000B6050F096AF60F02E3092AFCD70A0F10
:101A9000086E042E03D0FB0F01E3092A095000B0A1
:101AA000090F00B2080F00B4060F00B6020F00B80D
:101AB000050F0A6AF60F02E30A2AFCD70A0F096E1D
:101AC000042E03D0FB0F01E30A2A0A5000B0030FD3
:101AD00000B2070F00B4050F00B6010F00B8020FE7
:101AE00000BA050F0B6AF60F02E30B2AFCD70A0FA8
:101AF0000A6E042E03D0FB0F01E30B2A0B5000B03B
:101B0000050F00B4010F00B6030F00B8060F00BAAE
:101B1000020F00BC050F0C6AF60F02E30C2AFCD77B
:101B20000A0F0B6E042E03D0FB0F01E30C2A0C509E
:101B300000B0070F00B2050F00BA010F00BC020F82
:101B400000BE050F0D6AF60F02E30D2AFCD70A0F3F
:101B50000C6E042E03D0FB0F01E30D2A0D5000B0D4
:101B6000070F00B2050F00B4010F00B6020F00B856
:101B7000040F00BA080F00BC060F00BE020F01B030
:101B8000050F0E6AF60F02E30E2AFCD70A0F0D6E40
:101B9000042E03D0FB0F01E30E2A0E5000B0040FF9
:101BA00000B2090F00B4090F00B6080F00B8060F05
:101BB00000BA020F00BC050F00BE010F01B0020FFA
:101BC00001B2050F0F6AF60F02E30F2AFCD70A0FC6
:101BD0000E6E042E03D0FB0F01E30F2A0F5000B04E
:101BE000040F00B2080F00B4070F00B6050F00B8CD
:101BF000010F00BA030F00BC060F00BE030F01B0B7
:101C0000060F01B2020F01B4050F106AF60F02E3CE
:101C1000102AFCD70A0F0F6E042E03D0FB0F01E32E
:101C2000102A105000B0060F00B2020F00B4050FCA
:101C300000B6010F00B8030F00BA060F00BC020F78
:101C400000BE050F01B2010F01B4020F01B6050F6E
:101C5000116AF60F02E3112AFCD70A0F106E042E48
:101C600003D0FB0F01E3112A115000B0040F00B2A2
:101C7000090F00B4080F00B6070F00B8040F00BA30
:101C8000080F00BC070F00BE040F01B0090F01B21E
:101C9000080F01B4060F01B6020F01B8050F126A52
:101CA000F60F02E3122AFCD70A0F116E042E03D09E
:101CB000FB0F01E3122A125000B4010F00B6030F0C
:101CC00000B8070F00BA040F00BC090F00BE090FCF
:101CD00001B0080F01B2070F01B4050F01B6010FE3
:101CE00001B8020F01BA050F136AF60F02E3132AB7
:101CF000FCD70A0F126E042E03D0FB0F01E3132A48
:101D0000135000B0060F00B2020F00B4040F00B66B
:101D1000080F00B8060F00BA030F00BC060F00BE84
:101D2000030F01B0070F01B2050F01B4010F01B697
:101D3000030F01B8060F01BA020F01BC050F146AA8
:101D4000F60F02E3142AFCD70A0F136E042E03D0F9
:101D5000FB0F01E3142A145000B0090F00B2090F61
:101D600000B4080F00B6060F00B8030F00BA070F43
:101D700000BC040F00BE090F01B0080F01B2070F2D
:101D800001B4050F01BA010F01BC020F01BE050F1E
:101D9000156AF60F02E3152AFCD70A0F146E042EFB
:101DA00003D0FB0F01E3152A155000B0050F00B258
:101DB000010F00B4030F00B6070F00B8050F00BCF9
:101DC000010F00BE020F01B0050F01B2010F01B4F7
:101DD000030F01B6070F01B8040F01BA080F01BCC9
:101DE000060F01BE020F02B0050F166AF60F02E3DE
:101DF000162AFCD70A0F156E042E03D0FB0F01E341
:101E0000162A165000B2010F00B4020F00B6040FDC
:101E100000B8090F00BA090F00BC080F00BE060F7A
:101E200001B0020F01B2050F01B8010F01BA020F94
:101E300001BC050F01BE010F02B0020F02B2050F77
:101E4000176AF60F02E3172AFCD70A0F166E042E44
:101E500003D0FB0F01E3172A175000BA010F00BC93
:101E6000030F00BE070F01B0050F01B4010F01B64B
:101E7000020F01B8040F01BA080F01BC060F01BE22
:101E8000030F02B0060F02B2020F02B4050F186A68
:101E9000F60F02E3182AFCD70A0F176E042E03D0A0
:101EA000FB0F01E3182A185001B0010F01B2030F14
:101EB00001B4060F01B6020F01B8040F01BA080FF2
:101EC00001BC070F01BE050F02B2010F02B4020FE1
:101ED00002B6050F196AF60F02E3192AFCD70A0F9A
:101EE000186E042E03D0FB0F01E3192A195001B616
:101EF000010F01B8020F01BA040F01BC090F01BEA6
:101F0000090F02B0090F02B2080F02B4060F02B6A1
:101F1000020F02B8050F1A6AF60F02E31A2AFCD75D
:101F20000A0F196E042E03D0FB0F01E31A2A1A5070
:101F300001BE010F02B0030F02B2070F02B4050F7A
:101F400002B6010F02B8020F02BA050F1B6AF60FA4
:101F500002E31B2AFCD70A0F1A6E042E03D0FB0FD4
:101F600001E31B2A1B5002B4010F02B6030F02B893
:101F7000060F02BA020F02BC050F1C6AF60F02E33D
:101F80001C2AFCD70A0F1B6E042E03D0FB0F01E3A3
:101F90001C2A1C5002BA010F02BC020F02BE050F20
:101FA0001D6AF60F02E31D2AFCD70A0F1C6E042ED1
:101FB00003D0FB0F01E31D2A300FEE6E1B50300FD4
:101FC000EE6E1A50300FEE6E1950300FEE6E185044
:101FD000300FEE6E1750300FEE6E1650300FEE6E63
:101FE0001550300FEE6E1450300FEE6E1350300F50
:101FF000EE6E1250300FEE6E1150300FEE6E10502C
:10200000300FEE6E0F50300FEE6E0E50300FEE6E42
:102010000D50300FEE6E0C50300FEE6E0B50300F37
:10202000EE6E0A50300FEE6E0950300FEE6E085013
:10203000300FEE6E0750300FEE6E0650300FEE6E22
:102040000550300FEE6E170EE4CF1DF0E4CF1CF0FC
:10205000E4CF1BF0E4CF1AF0E4CF19F0E4CF18F08E
:10206000E4CF17F0E4CF16F0E4CF15F0E4CF14F08E
:10207000E4CF13F0E4CF12F0E4CF11F0E4CF10F08E
:10208000E4CF0FF0E4CF0EF0E4CF0DF0E4CF0CF08E
:10209000E4CF0BF0E4CF0AF0E4CF09F0E4CF08F08E
:1020A000E4CF07F0E4CF06F0E4CF05F0120000C063
:1020B000E5FF01C0E5FF02C0E5FF03C0E5FF05C085
:1020C000E5FFEBEC38F094928B922DEC35F0F3CFEA
:1020D00001F0F4CF02F0E9CF03F0880F04017C6F28
:1020E000130E01207D6F000E02207E6F000E032074
:1020F0007F6FB1EC2BF09284800E006E0F0E016E9C
:102100000F0E036E380E002603500122800E026E61
:102110000F0E036E800E005E0350015A0F0E056E07
:10212000380E0226055003220F0E056E800E025E49
:102130000550035A02C0E9FF03C0EAFFEFCF02F0E7
:10214000028400C0E9FF01C0EAFF02C0EFFF020EF7
:10215000E56E000EE56A68EC2FF0E652E6529386D3
:10216000810E006E0F0E016E0F0E036E380E0026EC
:10217000035001220F0E036E800E005E0350015AC1
:10218000810E026E0F0E036E0F0E056E380E0226C4
:10219000055003220F0E056E800E025E0550035A95
:1021A00002C0E9FF03C0EAFFEFCF02F0028600C0E1
:1021B000E9FF01C0EAFF02C0EFFF090EE56E010E64
:1021C000E56E68EC2FF0E652E652899A899089868E
:1021D0008982929A92909296929204019283800EB2
:1021E000006E040E016E0F0E036E380E00260350B3
:1021F00001220F0E036E800E005E0350015A800E06
:10220000026E040E036E0F0E056E380E0226055088
:1022100003220F0E056E800E025E0550035A02C0A7
:10222000E9FF03C0EAFFEFCF02F0029200C0E9FF2E
:1022300001C0EAFF02C0EFFF9283800E006E040E21
:10224000016E0F0E036E380E0026035001220F0E92
:10225000036E800E005E0350015A800E026E040E63
:10226000036E0F0E056E380E0226055003220F0E68
:10227000056E800E025E0550035A02C0E9FF03C0DE
:10228000EAFFEFCF02F0029200C0E9FF01C0EAFFCF
:1022900002C0EFFF9283800E006E040E016E0F0EDF
:1022A000036E380E0026035001220F0E036E800EBF
:1022B000005E0350015A800E026E040E036E0F0E74
:1022C000056E380E0226055003220F0E056E800E95
:1022D000025E0550035A02C0E9FF03C0EAFFEFCFD8
:1022E00002F0029200C0E9FF01C0EAFF02C0EFFF66
:1022F0000C0E0F01546F0F01549B54990F01556B35
:1023000092980401936B020E946F956B0A0E966F70
:10231000976B100E986F070E996F9A6B800EE56E93
:10232000040EE56EB60EE56E68EC30F0030EE126A5
:10233000800EE56E040EE56ED70EE56E48EC26F0D5
:10234000030EE126800EE56E040EE56EC60EE56E08
:1023500048EC26F0030EE1260401B16BB26BB36BBF
:10236000B46BB591B5959C6B9D6B9E6B9F6BA46B8D
:10237000A56BA66BA76B8A908A9A8A828A889390AB
:10238000939A9392939804019283800E006E040EA8
:10239000016E0F0E036E380E0026035001220F0E41
:1023A000036E800E005E0350015A800E026E040E12
:1023B000036E0F0E056E380E0226055003220F0E17
:1023C000056E800E025E0550035A02C0E9FF03C08D
:1023D000EAFFEFCF02F0029200C0E9FF01C0EAFF7E
:1023E00002C0EFFF9283800E006E040E016E0F0E8E
:1023F000036E380E0026035001220F0E036E800E6E
:10240000005E0350015A800E026E040E036E0F0E22
:10241000056E380E0226055003220F0E056E800E43
:10242000025E0550035A02C0E9FF03C0EAFFEFCF86
:1024300002F0029200C0E9FF01C0EAFF02C0EFFF14
:102440009283800E006E040E016E0F0E036E380E26
:102450000026035001220F0E036E800E005E035013
:10246000015A800E026E040E036E0F0E056E380EBA
:102470000226055003220F0E056E800E025E0550E7
:10248000035A02C0E9FF03C0EAFFEFCF02F0029255
:1024900000C0E9FF01C0EAFF02C0EFFF0C0EBD6EF5
:1024A000BD9ABD98BE6AB96AB98293940A01006B5D
:1024B000020E016F026B0A0E036F046B100E056FA4
:1024C000070E066F076B800EE56E0A0EE56E230E93
:1024D000E56E68EC30F0030EE126800EE56E0A0E24
:1024E000E56E440EE56E48EC26F0030EE126800E04
:1024F000E56E0A0EE56E330EE56E48EC26F0030E2F
:10250000E1260A011E6B1F6B206B216B2291229525
:10251000096B0A6B0B6B0C6B116B126B136B146BEF
:10252000E4CF05F0E4CF03F0E4CF02F0E4CF01F014
:10253000E4CF00F012004320502025640A0043003D
:102540002563000000C0E5FF01C0E5FF02C0E5FF14
:1025500003C0E5FF04C0E5FF05C0E5FF06C0E5FFD9
:1025600007C0E5FF08C0E5FF09C0E5FF0AC0E5FFB9
:102570000BC0E5FF006A016A040E015CD8B0E8D127
:102580000101102B100E105D01E3106B01011039D9
:10259000E8441F0B026E036A620E0226010E03223C
:1025A00002C0E9FF03C0EAFFEFCF02F0070E1015EB
:1025B000036E010E046E000E056E035006E0E86C1B
:1025C000D89004360536010FFCE3066A0250041663
:1025D00006500516045005E1055003E1046A042A7B
:1025E00001D0046A0450D880E866D890046A0436A2
:1025F0000450D8B4C1D701011051020DF450036E3C
:10260000F3CF02F0E00E0224046E000E0320056EEC
:1026100004C0E9FF05C0EAFFEECF04F0EFCF05F0FC
:1026200001010DA19DD0750E0224066E0A0E032035
:10263000076E06C0E9FF07C0EAFFEECF06F0EFCF56
:1026400007F00550800FF36E0750800FF35C02E136
:102650000650045C03E2046A056A60D0950E022607
:102660000A0E032202C0E9FF03C0EAFFEECF02F028
:10267000EFCF03F00350800FF36E0550800FF35C33
:1026800002E10450025C04E204683F0E056E46D08D
:102690000650045C086E07500558096EE86A09BECA
:1026A000FF0E0A6EE56E0A50E56E0950E56E0850A1
:1026B000E56EE56AE56A400EE56E000EE56A91ECAE
:1026C00022F0086EF3CF09F0F4CF0AF0E9CF0BF057
:1026D000080EE1260650025C066E07500358076E8E
:1026E000E86A07BEFF0E026EE56E0250E56E075007
:1026F000E56E0650E56E0B50E56E0A50E56E09502A
:10270000E56E0850E56E16EC29F0026EF3CF03F08B
:10271000080EE1260250046E0350056E01010C51B3
:10272000800FF36E0550800FF35C02E104500B5DE7
:1027300003E3046A056A14D001010B51FF08026E1D
:102740003F0E0C55036E0550800FF36E0350800F43
:10275000F35C02E10250045C03E304683F0E056E83
:1027600001011051020DF450036EF3CF02F0550E2B
:1027700002260A0E032202C0E9FF03C0EAFFEECFE1
:1027800002F0EFCF03F00250045C026E03500558D4
:10279000036ED88003AED89004E3031E026CD8B455
:1027A000032A012A01010C51800FF36E0350800FA0
:1027B000F35C02E102500B5DD8B0DED6010110518E
:1027C000020DF450076EF3CF06F0550E06260A0EE2
:1027D000072206C0E9FF07C0EAFF04C0EEFF05C0FC
:1027E000EFFF01010DA55AD001011051020DF45067
:1027F000076EF3CF06F0B50E0624086E0A0E07200A
:10280000096E08C0E9FF09C0EAFFEECF0AF0EFCF7A
:102810000BF00A500B10D8B441D05C0E0626040E03
:10282000072206C0E9FF07C0EAFFEECF06F0EFCFB0
:1028300007F00650045C026E07500558036E021044
:102840001CE00350800F800F02E1010E025C066A5B
:1028500006360B50800F800F02E1010E0A5C0A6AF7
:102860000A3606500A1809E108C0E9FF09C0EAFF64
:1028700002C0EEFF03C0EFFF7FD601011051020D31
:10288000F450036EF3CF02F0B50E02260A0E0322B7
:1028900002C0E9FF03C0EAFFEE6AEF6A01010DA37F
:1028A00043D000500EE100C002F0002A036A110E6E
:1028B0000226010E032202C0E9FF03C0EAFF420E16
:1028C000EF6E00C002F0002A036A110E0226010E0C
:1028D0000322640E01011025066E02C0E9FF03C049
:1028E000EAFF06C0EFFF00C002F0002A036A110EE3
:1028F0000226010E03220550066E02C0E9FF03C046
:10290000EAFF06C0EFFF00C002F0002A036A110EC2
:102910000226010E03220450066E02C0E9FF03C026
:10292000EAFF06C0EFFF28D610C102F00550E56EA1
:102930000450E56EE56A0250E56E000EE56E580E35
:10294000E56E4A0EE56E24EC32F0070EE12614D651
:1029500000501DE001010DA31AD000C002F0002AB2
:10296000036A110E0226010E032202C0E9FF03C012
:10297000EAFF0A0EEF6E0050E56E800EE56E010E66
:10298000E56E110EE56E36EC2BF0040EE1260150DB
:10299000E4CF0BF0E4CF0AF0E4CF09F0E4CF08F085
:1029A000E4CF07F0E4CF06F0E4CF05F0E4CF04F085
:1029B000E4CF03F0E4CF02F0E4CF01F0E4CF00F085
:1029C000120000C0E5FF01C0E5FF02C0E5FF03C043
:1029D000E5FFFCEC27F052EC20F02DEC35F0006E1A
:1029E000F3CF01F0F4CF02F0E9CF03F004017C5102
:1029F000005E7D51015A7E51025A7F51035A039E57
:102A00003F0E035C08E1FF0E025C05E1FF0E015C76
:102A100002E1FF0E005CD8B00DEF17F02DEC35F0A1
:102A2000F3CF01F0F4CF02F0E9CF03F0880F0401F7
:102A30007C6F130E01207D6F000E02207E6F000E52
:102A400003207F6FA2EC12F004C0E5FFF2CF04F088
:102A5000F29E0401A95101012C6F0401AA51010148
:102A60002D6F0401AB5101012E6F0401AC51010126
:102A70002F6F0401AD510101306F0401AE5101010E
:102A8000316F0401AF510101326F0401B0510101F6
:102A9000336F0401B1510101346F0401B2510101DE
:102AA000356F0401B3510101366F0401B4510101C6
:102AB000376F0401B5510101386F0401AD6BAE6B86
:102AC000AF6BB06B04BEF28EE4CF04F0800EE56E07
:102AD000040EE56E930EE56E44EC09F0030EE1265C
:102AE0009EC468F19FC469F101016951800F7C0F98
:102AF00002E1000E685D04E301016869030E696F7D
:102B000001016951800F840F02E1010E685D05E249
:102B1000010E0101686FFC0E696F01016951800FA0
:102B2000800F02E1010E685D10E301016951800F21
:102B3000F36E04019751800FF35C03E1965101019C
:102B4000685D03E20101686B696BD880010169AFC0
:102B5000D89015E30401971D016E961D006E004A82
:102B6000012A0150800FF36E01016951800FF35C5F
:102B700002E16851005C03E20101686B696B0401CA
:102B8000B5A507D0D880010169AFD89002E3686B82
:102B9000696BD880010169AFD89007E3691D016EA8
:102BA000681D006E004A012A04D068C100F069C1A6
:102BB00001F000C06AF101C06BF101016A51020B22
:102BC000E840010BE838E844F46E0F015451DF0B84
:102BD000F410546F01016A51010B010BE838F46ED7
:102BE0000F015451EF0BF410546F01016B356B3131
:102BF000016E6A31006E01340132003200500F0163
:102C0000556FD880010169AFD89003E3899A898014
:102C100002D08990898A04C0E5FFF2CF04F0F29EC9
:102C20000A01165101012C6F0A01175101012D6F84
:102C30000A01185101012E6F0A01195101012F6F6C
:102C40000A011A510101306F0A011B510101316F54
:102C50000A011C510101326F0A011D510101336F3C
:102C60000A011E510101346F0A011F510101356F24
:102C70000A0120510101366F0A0121510101376F0C
:102C80000A0122510101386F0A011A6B1B6B1C6B80
:102C90001D6B04BEF28EE4CF04F0800EE56E0A0ECA
:102CA000E56E000EE56E44EC09F0030EE1260BCA5A
:102CB00068F10CCA69F101016951800F7C0F02E1D2
:102CC000000E685D04E301016869030E696F01018C
:102CD0006951800F840F02E1010E685D05E2010E6B
:102CE0000101686FFC0E696F01016951800F800F4F
:102CF00002E1010E685D10E301016951800FF36E7E
:102D00000A010451800FF35C03E103510101685D86
:102D100003E20101686B696BD880010169AFD8904B
:102D200015E30A01041D016E031D006E004A012A0D
:102D30000150800FF36E01016951800FF35C02E1D5
:102D40006851005C03E20101686B696B0A0122A50E
:102D500007D0D880010169AFD89002E3686B696B36
:102D6000D880010169AFD89007E3691D016E681D25
:102D7000006E004A012A04D068C100F069C101F068
:102D800000C06AF101C06BF101016A51020BE84019
:102D9000010BE838E844F46EBD50DF0BF410BD6E53
:102DA0006A51010B010BE838F46EBD50EF0BF410C3
:102DB000BD6E6B356B31016E6A31006E01340132CC
:102DC00000320050BE6ED880010169AFD89003E395
:102DD0008A908A8A02D08A9A8A8000C100F001C152
:102DE00001F00101003F01D0012B0050140A02E163
:102DF000015001E012D00101006B016B04019F51F1
:102E0000E56E9E51E56E000EE56E250EE56E360E02
:102E1000E56E24EC32F0050EE126E4CF03F0E4CFBA
:102E200002F0E4CF01F0E4CF00F01200D9CFE5FFCB
:102E3000E1CFD9FF00C0E5FF01C0E5FF02C0E5FF1B
:102E400003C0E5FF04C0E5FF05C0E5FF06C0E5FFE0
:102E500007C0E5FF08C0E5FF09C0E5FF0AC0E5FFC0
:102E60000BC0E5FF020EDBCF00F0030EDBCF01F05D
:102E7000040EDBCF02F0050EDBCF03F0060EDBCF36
:102E800004F002500A6E0150096E0050086EE56AA7
:102E9000110EE56E0A50E56E0950E56E0850E56EBC
:102EA000800EE56E040EE56E240EE56EB4EC2AF09D
:102EB000080EE12633C405F034C406F0E86A0401C4
:102EC00034BFFF0E076E0101406F06503F6F055083
:102ED0003E6F3D6B03C005F004C006F0E86A04BE17
:102EE000FF0E076E086E24C409F0E56AE56AE56A1C
:102EF0000950E56E0850E56E0750E56E0650E56E28
:102F00000550E56E91EC22F00101396FF3CF3AF1F3
:102F1000F4CF3BF1E9CF3CF1080EE1260401255145
:102F2000D8B4AFD00450800F800F02E1010E035CD3
:102F300025E304012A51800F7C0F08E1000E295D72
:102F400005E1000E285D02E1000E275D17E2040195
:102F50003251800FF36E01014051800FF35C0DE19F
:102F60003F510401315D09E101013E510401305D31
:102F700004E101013D5104012F5D33E3D88004AE2B
:102F8000D890D8A043D004012A51800F840F08E1C3
:102F9000000E295D05E1000E285D02E1010E275DAE
:102FA00035E30101401D0A6E3F1D096E3E1D046E92
:102FB0003D1D036E032A04E1042A02E1094A0A2A9C
:102FC0000A50800FF36E04013251800FF35C08E168
:102FD0003151095C05E13051045C02E12F51035C81
:102FE00015E2055004012725036E06502821046EC2
:102FF00007502921096E08502A210A6E0350276FB5
:103000000450286F0950296F0A502A6F040127398C
:103010000F0B036E2839046EF00B041A0326295196
:10302000E838F00B041229390F0B096E2A390A6EA1
:10303000F00B0A1A0926F00E0AB60A2625C40BF070
:10304000E56AE56AE56A0B50E56E0A50E56E0950DF
:10305000E56E0450E56E0350E56E91EC22F0036ED0
:10306000F3CF04F0F4CF09F0E9CF0AF0080EE1261F
:1030700003500101392704503A2309503B230A50D9
:103080003C2304012651D8B46CD02B51055C0101BE
:10309000416F04012C5106580101426F04012D516A
:1030A00007580101436F04012E5108580101446F74
:1030B000800F800F08E1010E435D05E1000E425DC7
:1030C00002E1000E415D07E3FF0E0101416F426F17
:1030D000436B446B14D001014451800F810F08E110
:1030E000FF0E435D05E1000E425D02E1000E415D11
:1030F00006E20101416B426BFF0E436F446F010119
:10310000443143310A6E096A09324251E8407F0B6B
:10311000091242314131046E036A033226C40BF0B6
:10312000E56AE56AE56A0B50E56E0A50E56E0950FE
:10313000E56E0450E56E0350E56E91EC22F0036EEF
:10314000F3CF04F0F4CF09F0E9CF0AF0080EE1263E
:1031500003500101392704503A2309503B230A50F8
:103160003C23055004012B6F06502C6F07502D6F28
:1031700008502E6F01014051800FF36E01013C5148
:10318000800FF35C0DE13B5101013F5D09E101015D
:103190003A5101013E5D04E10101395101013D5DFA
:1031A00011E201013D5104012F6F01013E51040163
:1031B000306F01013F510401316F010140510401A1
:1031C000326F3AD00101401D066E3F1D056E3E1D57
:1031D000046E3D1D036E032A04E1042A02E1054A40
:1031E000062A01013C51800FF36E0650800FF35CFC
:1031F00008E105503B5D05E104503A5D02E10350F2
:10320000395D0AE2035004012F6F0450306F0550FE
:10321000316F0650326F10D00101395104012F6F08
:1032200001013A510401306F01013B510401316F3A
:1032300001013C510401326FE56A110EE56E800E0A
:10324000E56E040EE56E240EE56E0250E56E01504B
:10325000E56E0050E56EB4EC2AF0080EE126E4CFEE
:103260000BF0E4CF0AF0E4CF09F0E4CF08F0E4CFAC
:1032700007F0E4CF06F0E4CF05F0E4CF04F0E4CFAC
:1032800003F0E4CF02F0E4CF01F0E4CF00F0E4CFAC
:10329000D9FF1200D9CFE5FFE1CFD9FF00C0E5FF8C
:1032A00001C0E5FF02C0E5FF03C0E5FF04C0E5FF84
:1032B00005C0E5FF06C0E5FF07C0E5FF08C0E5FF64
:1032C00009C0E5FF0AC0E5FF020EDBCF00F0030EE8
:1032D000DBCF01F0040EDBCF02F0036A046A57EC87
:1032E00035F0056EFE0A01E078D014EC30F057ECB2
:1032F00035F0066E030E065CD8A05BD0060E065CA9
:10330000D8B057D0FD0E0624076EFA6AFB6A073460
:10331000FA36E834FA36FC0B280FE56E330EFA2243
:10332000000EFB22E450F96E9AEF19F0ACEF19F0A1
:10333000C5EF19F00050090F076E000E0120086E4E
:10334000000E022007C0E9FF08C0F3FFC4EC37F00D
:10335000036EF3CF04F02DD00050090F076E000E5E
:103360000120086E000E0220096E020E0726000ED4
:103370000822092207C0E9FF08C0F3FF0950C4EC86
:1033800037F0036EF3CF04F014D00050070F076E30
:10339000000E0120086E000E022007C0E9FF08C0E1
:1033A000F3FF29EC38F0076E07C003F0046A07BE8C
:1033B000046806C007F00450E56E0350E56EE56A48
:1033C0000750E56E000EE56E190EE56EA40EE56E73
:1033D00024EC32F0070EE1262BD1070E055CD8B0A5
:1033E00027D1FA6AFB6A0534FA36E834FA36FC0B60
:1033F000000FE56E340EFA22000EFB22E450F96E47
:103400000EEF1AF029EF1AF03BEF1AF04DEF1AF019
:103410007FEF1AF0B5EF1AF0CBEF1AF00050230F40
:10342000036E000E0120046E000E0220E56E0450B3
:10343000E56E0350E56E87EC1CF0030EE126020EEC
:10344000E56E00C0E9FF01C0F3FF0250B7EC38F0B1
:10345000EFD00050330F036E000E0120046E000EFB
:103460000220E56E0450E56E0350E56E14EC1FF08B
:10347000030EE126DDD00050440F036E000E012044
:10348000046E000E0220E56E0450E56E0350E56EFA
:1034900014EC1FF0030EE126CBD00050090F036E91
:1034A000000E0120046E000E0220056E57EC35F070
:1034B0000A6E096AE56A0AC0F4FF03C0E9FF04C0A6
:1034C000F3FF055094EC38F057EC35F0086A092604
:1034D00008500A2209C0E5FF0AC0F4FF03C0E9FF53
:1034E00004C0F3FF055094EC38F0010EE56E00C007
:1034F000E9FF01C0F3FF0250B7EC38F099D000505B
:10350000090F036E000E0120046E000E0220056EEE
:10351000020E0326000E0422052257EC35F00A6E37
:10352000096AE56A0AC0F4FF03C0E9FF04C0F3FFBB
:10353000055094EC38F057EC35F0086A092608502D
:103540000A2209C0E5FF0AC0F4FF03C0E9FF04C076
:10355000F3FF055094EC38F0E56A00C0E9FF01C0C4
:10356000F3FF0250B7EC38F063D00050070F036E42
:10357000000E0120046E000E0220056E57EC35F09F
:10358000076E07C0E5FF03C0E9FF04C0F3FF055065
:10359000B7EC38F04DD057EC35F0066E0050160FF2
:1035A000036E000E0120046E000E0220056E035013
:1035B0000C0F076E000E0420086E000E0520096E29
:1035C0000650010BF46E07C0E9FF08C0F3FF095075
:1035D00029EC38F0FE0BF410E56E07C0E9FF08C0D7
:1035E000F3FF0950B7EC38F00650010A21E1080E4C
:1035F0000326000E04220522E56AF46AF66AF76AD9
:1036000003C0E9FF04C0F3FF05503AEC38F0230E85
:103610000026000E01220222E56AE56A0250E56EEC
:103620000150E56E0050E56E89EC28F0050EE126AC
:10363000E4CF0AF0E4CF09F0E4CF08F0E4CF07F0DC
:10364000E4CF06F0E4CF05F0E4CF04F0E4CF03F0DC
:10365000E4CF02F0E4CF01F0E4CF00F0E4CFD9FFF3
:10366000120000C0E5FF01C0E5FF02C0E5FF03C096
:10367000E5FF04C0E5FF05C0E5FF06C0E5FF07C0A4
:10368000E5FF08C0E5FF09C0E5FF0AC0E5FF0BC084
:10369000E5FF0CC0E5FF0DC0E5FF0EC0E5FF000E25
:1036A00000B0010F00B2020F00B4040F00B6080F03
:1036B00000B8060F00BA020F00BC040F00BE080FCE
:1036C00001B0060F01B2020F01B4040F01B6080FDA
:1036D00001B8060F01BA020F01BC040F01BE080FAA
:1036E00002B0060F02B2020F02B4040F02B6080FB6
:1036F00002B8060F02BA020F02BC040F02BE080F86
:10370000056AF60F02E3052AFCD70A0F046E05507E
:1037100000B8010F00BA030F00BC060F00BE020F75
:1037200001B0050F01B2010F01B4020F01B6040F81
:1037300001B8090F01BA090F01BC080F01BE060F3D
:1037400002B0030F02B2070F02B4040F02B6080F53
:1037500002B8070F02BA050F066AF60F02E3062A3F
:10376000FCD70A0F056E065000BE010F01B0020F14
:1037700001B2050F01BA010F01BC030F01BE070F13
:1037800002B0050F02B4010F02B6020F02B8050F16
:1037900002BA010F02BC030F02BE060F076AF60F42
:1037A00002E3072AFCD70A0F066E075001B4010F87
:1037B00001B6020F01B8040F01BA080F01BC060FD1
:1037C00001BE020F02B0050F02B2010F02B4020FD8
:1037D00002B6040F02B8080F02BA070F02BC040FAA
:1037E00002BE080F086AF60F02E3082AFCD70A0F88
:1037F000076E085001BC010F01BE030F02B0060F97
:1038000002B2030F02B4060F02B6020F02B8040F91
:1038100002BA090F02BC090F02BE080F096AF60FAF
:1038200002E3092AFCD70A0F086E095002B2010F01
:1038300002B4020F02B6050F02BC010F02BE030F55
:103840000A6AF60F02E30A2AFCD70A0F096E0A5029
:1038500002B8010F02BA020F02BC040F02BE080F29
:103860000B6AF60F02E30B2AFCD70A0F0A6E0B5005
:103870000E6A0EE10A5010E1095012E1085014E1FD
:10388000075016E1065018E105501AE104501CD00B
:103890000E2A300FEE6E0A500E2A300FEE6E0950CF
:1038A0000E2A300FEE6E08500E2A300FEE6E0750C3
:1038B0000E2A300FEE6E06500E2A300FEE6E0550B7
:1038C0000E2A300FEE6E04500E2A300FEE6E0E50A0
:1038D000E4CF0EF0E4CF0DF0E4CF0CF0E4CF0BF02A
:1038E000E4CF0AF0E4CF09F0E4CF08F0E4CF07F02A
:1038F000E4CF06F0E4CF05F0E4CF04F0E4CF03F02A
:10390000E4CF02F0E4CF01F0E4CF00F01200D9CF11
:10391000E5FFE1CFD9FF00C0E5FF01C0E5FF02C030
:10392000E5FF03C0E5FF04C0E5FF05C0E5FF06C0F5
:10393000E5FF07C0E5FF08C0E5FF09C0E5FF0AC0D5
:10394000E5FF0BC0E5FF020EDBCF00F0030EDBCF7F
:1039500001F0040EDBCF02F0036A046A57EC35F085
:10396000056EFE0A01E063D014EC30F057EC35F040
:10397000066E06500AE00650010A19E00650020AD7
:1039800028E006500A0A37E040D00050060F076EC4
:10399000000E0120086E000E022007C0E9FF08C0DB
:1039A000F3FFC4EC37F0036EF3CF04F02ED00050D9
:1039B0000C0F076E000E0120086E000E022007C0DB
:1039C000E9FF08C0F3FFC4EC37F0036EF3CF04F057
:1039D0001CD000500E0F076E000E0120086E000E66
:1039E000022007C0E9FF08C0F3FFC4EC37F0036E04
:1039F000F3CF04F00AD000C0E9FF01C0F3FF02508A
:103A0000C4EC37F0036EF3CF04F00450E56E0350BE
:103A1000E56EE56A0650E56E000EE56E610EE56E38
:103A20006E0EE56E24EC32F0070EE126A1D00550B3
:103A30000CE00550010A32E00550020A01E157D0BE
:103A400005500A0A01E17CD093D00050060F056EA4
:103A5000000E0120066E000E0220076E57EC35F0B6
:103A60000B6E0A6AE56A0BC0F4FF05C0E9FF06C0E9
:103A7000F3FF075094EC38F057EC35F0096A0A264A
:103A800009500B220AC0E5FF0BC0F4FF05C0E9FF97
:103A900006C0F3FF075094EC38F06AD000500C0FCA
:103AA000056E000E0120066E000E0220076E57EC18
:103AB00035F00B6E0A6AE56A0BC0F4FF05C0E9FF3A
:103AC00006C0F3FF075094EC38F057EC35F0096A64
:103AD0000A2609500B220AC0E5FF0BC0F4FF05C0FF
:103AE000E9FF06C0F3FF075094EC38F041D00050D6
:103AF0000E0F056E000E0120066E000E0220076EEE
:103B000057EC35F00B6E0A6AE56A0BC0F4FF05C08E
:103B1000E9FF06C0F3FF075094EC38F057EC35F09E
:103B2000096A0A2609500B220AC0E5FF0BC0F4FF00
:103B300005C0E9FF06C0F3FF075094EC38F018D039
:103B400057EC35F0046E036A57EC35F0066A03262D
:103B5000065004220450E56E0350E56E0250E56EF7
:103B60000150E56E0050E56E06EC34F0050EE126DE
:103B7000E4CF0BF0E4CF0AF0E4CF09F0E4CF08F093
:103B8000E4CF07F0E4CF06F0E4CF05F0E4CF04F093
:103B9000E4CF03F0E4CF02F0E4CF01F0E4CF00F093
:103BA000E4CFD9FF1200800EE56E0A0EE56E950E89
:103BB000E56EBBEC30F0030EE126800EE56E0A0EDA
:103BC000E56E750EE56EBBEC30F0030EE126800E5F
:103BD000E56E0A0EE56E970EE56EBBEC30F0030E57
:103BE000E126800EE56E0A0EE56E770EE56EBBEC03
:103BF00030F0030EE126800EE56E0A0EE56E990E9A
:103C0000E56EBBEC30F0030EE126800EE56E0A0E89
:103C1000E56E790EE56EBBEC30F0030EE126800E0A
:103C2000E56E0A0EE56E9B0EE56EBBEC30F0030E02
:103C3000E126800EE56E0A0EE56E7B0EE56EBBECAE
:103C400030F0030EE126800EE56E0A0EE56E9D0E45
:103C5000E56EBBEC30F0030EE126800EE56E0A0E39
:103C6000E56E7D0EE56EBBEC30F0030EE126800EB6
:103C7000E56E0A0EE56E9F0EE56EBBEC30F0030EAE
:103C8000E126800EE56E0A0EE56E7F0EE56EBBEC5A
:103C900030F0030EE126800EE56E0A0EE56EA10EF1
:103CA000E56EBBEC30F0030EE126800EE56E0A0EE9
:103CB000E56E810EE56EBBEC30F0030EE126800E62
:103CC000E56E0A0EE56EA30EE56EBBEC30F0030E5A
:103CD000E126800EE56E0A0EE56E830EE56EBBEC06
:103CE00030F0030EE126800EE56E0A0EE56EA50E9D
:103CF000E56EBBEC30F0030EE126800EE56E0A0E99
:103D0000E56E850EE56EBBEC30F0030EE126800E0D
:103D1000E56E0A0EE56EA70EE56EBBEC30F0030E05
:103D2000E126800EE56E0A0EE56E870EE56EBBECB1
:103D300030F0030EE126800EE56E0A0EE56EA90E48
:103D4000E56EBBEC30F0030EE126800EE56E0A0E48
:103D5000E56E890EE56EBBEC30F0030EE126800EB9
:103D6000E56E0A0EE56EAB0EE56EBBEC30F0030EB1
:103D7000E126800EE56E0A0EE56E8B0EE56EBBEC5D
:103D800030F0030EE126800EE56E0A0EE56EAD0EF4
:103D9000E56EBBEC30F0030EE126800EE56E0A0EF8
:103DA000E56E8D0EE56EBBEC30F0030EE126800E65
:103DB000E56E0A0EE56EAF0EE56EBBEC30F0030E5D
:103DC000E126800EE56E0A0EE56E8F0EE56EBBEC09
:103DD00030F0030EE126800EE56E0A0EE56EB10EA0
:103DE000E56EBBEC30F0030EE126800EE56E0A0EA8
:103DF000E56E910EE56EBBEC30F0030EE126800E11
:103E0000E56E0A0EE56EB30EE56EBBEC30F0030E08
:103E1000E126800EE56E0A0EE56E930EE56EBBECB4
:103E200030F0030EE1261200D9CFE5FFE1CFD9FF34
:103E300000C0E5FF01C0E5FF02C0E5FF03C0E5FFEC
:103E400004C0E5FF05C0E5FF06C0E5FF07C0E5FFCC
:103E500008C0E5FF020EDBCF00F0030EDBCF01F060
:103E6000040EDBCF02F0036A046A57EC35F0056EEE
:103E7000FE0A01E075D014EC30F057EC35F0066E18
:103E8000040E065CD8B05AD0FA6AFB6A0634FA36D9
:103E9000E834FA36FC0BA60FE56E3E0EFA22000E51
:103EA000FB22E450F96E5BEF1FF067EF1FF07AEF33
:103EB0001FF08DEF1FF000C0E9FF01C0F3FF0250BB
:103EC00029EC38F0076E07C003F0046A37D00050C1
:103ED000010F076E000E0120086E000E022007C0C1
:103EE000E9FF08C0F3FF29EC38F0076E07C003F0C4
:103EF000046A24D00050020F076E000E0120086EE5
:103F0000000E022007C0E9FF08C0F3FF29EC38F0DB
:103F1000076E07C003F0046A11D000500F0F076E40
:103F2000000E0120086E000E022007C0E9FF08C045
:103F3000F3FFC4EC37F0036EF3CF04F00450E56EEA
:103F40000350E56EE56A0650E56E000EE56E4D0E17
:103F5000E56EB00EE56E24EC32F0070EE1268DD052
:103F6000040E055CD8B089D0FA6AFB6A0534FA36CB
:103F7000E834FA36FC0B860FE56E3F0EFA22000E8F
:103F8000FB22E450F96ECBEF1FF0D8EF1FF003EFE8
:103F900020F019EF20F057EC35F0036E03C0E5FF79
:103FA00000C0E9FF01C0F3FF0250B7EC38F065D064
:103FB0000050010F036E000E0120046E000E02205F
:103FC000056E57EC35F0066E06C0E5FF03C0E9FF4D
:103FD00004C0F3FF0550B7EC38F00650D8A44DD01C
:103FE0000050030F036E000E0120046E000E02202D
:103FF000E56AF46AF66AF76A03C0E9FF04C0F3FFF2
:104000003AEC38F03AD00050020F036E000E012057
:10401000046E000E0220056E57EC35F0066E06C0E9
:10402000E5FF03C0E9FF04C0F3FF0550B7EC38F02B
:1040300024D00F0E0026000E0122022257EC35F08C
:10404000066E056AE56A06C0F4FF00C0E9FF01C01C
:10405000F3FF025094EC38F057EC35F0046A052673
:104060000450062205C0E5FF06C0F4FF00C0E9FFCA
:1040700001C0F3FF025094EC38F0E4CF08F0E4CF35
:1040800007F0E4CF06F0E4CF05F0E4CF04F0E4CF8E
:1040900003F0E4CF02F0E4CF01F0E4CF00F0E4CF8E
:1040A000D9FF120000C0E5FF01C0E5FF02C0E5FF37
:1040B00003C0E5FF04C0E5FF05C0E5FF06C0E5FF5E
:1040C00007C0E5FF08C0E5FF09C0E5FFC2B202D1A5
:1040D00001010F51D8B4ADD001010E51020DF450C1
:1040E000016EF3CF00F0E00E0026000E012200C0AA
:1040F000E9FF01C0EAFFEECF02F0EFCF03F0033497
:104100000330056E0230046E053405320432053486
:10411000053204320450025C046E05500358056EEB
:10412000C3CF06F0076A0650042607500522C4CF05
:1041300006F00650096E086A085004260950052248
:1041400000C0E9FF01C0EAFF04C0EEFF05C0EFFFB9
:1041500001010A51010A01E06AD001010E51020D6C
:10416000F450016EF3CF00F0E00E0024046E000E58
:104170000120056E04C0E9FF05C0EAFFEECF02F0A2
:10418000EFCF03F0750E00260A0E012200C0E9FFF2
:1041900001C0EAFFEECF04F0EFCF05F09C0E04263D
:1041A000D8A005060350800FF36E0550800FF35C16
:1041B00002E10450025C0EE20250640F046E000E35
:1041C0000320056E00C0E9FF01C0EAFF04C0EEFF56
:1041D00005C0EFFF01010E51020DF450016EF3CF47
:1041E00000F0950E00260A0E012200C0E9FF01C072
:1041F000EAFFEECF04F0EFCF05F0640E0426D8B04E
:10420000052A0550800FF36E0350800FF35C02E126
:104210000250045C0CE29C0E0226D8A0030600C0EB
:10422000E9FF01C0EAFF02C0EEFF03C0EFFF01019A
:104230000F6B01010E2B100E0E5D01E30E6B0101E1
:104240000E39E8441F0B006E016A620E0026010E53
:10425000012200C0E9FF01C0EAFFEFCF00F0070E26
:104260000E15016E010E026E000E036E015006E087
:10427000E86CD89002360336010FFCE3046A005064
:10428000021604500316025005E1035003E1026ACE
:10429000022A01D0026A0250D880E866D890026AE9
:1042A0000236025017E0230E01010E25006E016A4E
:1042B0000F0E012200C0E9FF01C0EAFFEFCF00F0BE
:1042C0000044E844FC0B016E0128C26EC282010E5C
:1042D00001010F6FE4CF09F0E4CF08F0E4CF07F05D
:1042E000E4CF06F0E4CF05F0E4CF04F0E4CF03F030
:1042F000E4CF02F0E4CF01F0E4CF00F01200D9CF18
:10430000E5FFE1CFD9FF00C0E5FF01C0E5FF02C036
:10431000E5FF03C0E5FF04C0E5FF05C0E5FF06C0FB
:10432000E5FF07C0E5FF08C0E5FF09C0E5FF0AC0DB
:10433000E5FF0BC0E5FF020EDBCF00F0030EDBCF85
:1043400001F0040EDBCF02F0050EDBCF03F0060E0A
:10435000DBCF04F0070EDBCF05F0080EDBCF06F055
:10436000090EDBCF07F006C008F0060608500EE085
:1043700006500424086EE86A06BEE8680520096E47
:1043800008C0E9FF09C0EAFFEF6AEDD7005001015C
:10439000596F01505A6F02505B6F03505C6F59C1E7
:1043A00000F05AC101F05BC102F05CC103F0066A83
:1043B000086A096A800E03140A6E065007E1085065
:1043C00005E1095003E10A50800A01E012D0039E82
:1043D00000500101596F01505A6F02505B6F03503A
:1043E0005C6F04C0E9FF05C0EAFF2D0EEF6E044AC2
:1043F000052A01015B355C357E08006E5951016E5E
:104400005A51026E7F0E5B15036E066A038E086AB0
:10441000096A0A6A0B6A005019E0D88000AED89089
:104420000EE30850082609360A360B3603BE08800C
:1044300001500126023603360636002AECD7D89002
:1044400006320332023201320006E5D70850091065
:104450000A100B1012E00550E56E0450E56E0B508B
:10446000E56E0A50E56E0950E56E0850E56E02EC07
:1044700035F0006E060EE12608D004C0E9FF05C045
:10448000EAFF300EEF6E010E006E00500426E86A5F
:1044900000BEE8680522075028E004C0E9FF05C017
:1044A000EAFF2E0EEF6E002A044A052A075018086C
:1044B000E56E0550E56E0450E56E0650E56E03505E
:1044C000E56E0250E56E0150E56E6FEC34F0016E62
:1044D000070EE1260150002607500426E86A05224F
:1044E00004C0E9FF05C0EAFFEF6A0050E4CF0BF01B
:1044F000E4CF0AF0E4CF09F0E4CF08F0E4CF07F00E
:10450000E4CF06F0E4CF05F0E4CF04F0E4CF03F00D
:10451000E4CF02F0E4CF01F0E4CF00F0E4CFD9FF24
:104520001200D9CFE5FFE1CFD9FF00C0E5FF01C000
:10453000E5FF02C0E5FF03C0E5FF04C0E5FF05C0DD
:10454000E5FF06C0E5FF07C0E5FF020EDBCF00F088
:10455000030EDBCF01F0040EDBCF02F0050EDBCF44
:1045600003F0060EDBCF04F0070EDBCF05F0080EDC
:10457000DBCF06F0090EDBCF07F000500101456FDD
:104580000150466F0250476F0350486F04500101BD
:10459000496F05504A6F06504B6F07504C6F010131
:1045A000455101014B03F4CF01F0F3CF00F000506F
:1045B00001014F6F0150506F010145510101490345
:1045C000F4CF01F0F3CF00F0005001014D6F015026
:1045D0004E6F0101485101014903F3CF00F0010181
:1045E000505100260050506F0101475101014A030C
:1045F000F3CF00F00101505100260050506F01012F
:10460000475101014903F4CF01F0F3CF00F001015C
:104610004F5100265051012200504F6F0150506FF2
:104620000101465101014A03F4CF01F0F3CF00F03C
:1046300001014F5100265051012200504F6F01508F
:10464000506F0101465101014B03F3CF00F00050C0
:104650000101546F0101465101014903F4CF01F0FA
:10466000F3CF00F000500101526F0150536F010170
:10467000455101014C03F3CF00F000500101586F88
:104680000101455101014A03F4CF01F0F3CF00F0DD
:1046900000500101566F0150576F0101516B01012C
:1046A000556B0101515101014D25006E010152511F
:1046B00001014E21016E0101535101014F21026E92
:1046C0000101545101015021036E00504D6F015002
:1046D0004E6F02504F6F0350506F01015551010151
:1046E0004D25006E0101565101014E21016E01015F
:1046F000575101014F21026E010158510101502112
:10470000036E03C0E9FF02C0F4FF01C0F3FF0050D5
:10471000E4CF07F0E4CF06F0E4CF05F0E4CF04F0F7
:10472000E4CF03F0E4CF02F0E4CF01F0E4CF00F0F7
:10473000E4CFD9FF120000C0E5FF01C0E5FF010191
:104740000751D8B4F5D09DA81DD09EA81BD001015B
:1047500076510101731905E178EC38F00101736BB2
:10476000E7D0000E01017625006E016A0F0E0122CE
:1047700000C0E9FF01C0EAFFEFCF6FF1762B6FC1F8
:10478000ADFFD6D09EAAD4D0ABA205D001017481D2
:1047900078EC38F0CDD0ABA405D00101748378EC6F
:1047A00038F0C6D0ABA03ED0AECF6FF1800E010185
:1047B000081101016F1904E101017489AB96B8D0A9
:1047C00001016F5104E06F510101081927E1010156
:1047D0007499AB9601016F5103E00101749702D007
:1047E000010174876FC178F171C179F1010171051F
:1047F00001017A6F600E01017925006E016A000ED9
:10480000012200C0E9FF01C0EAFF6FC1EFFF792B71
:104810007951800A02E10101796B8AD00101749912
:10482000AB8686D0AECF6FF1010174A919D0800E8E
:104830000101081101016F1911E18B909D9AAB984C
:104840000101735104E1AD6A78EC38F007D000CF74
:10485000ADFF010E0101766F9D886AD0AB8668D0EE
:1048600001016F51010178270101795101017A1984
:104870001BE1010178510CE179C171F1010174B7BB
:1048800012D08B909D9AAB98AD6A78EC38F00BD033
:104890000101748574B707D08B909D9AAB98010E77
:1048A000AD6E78EC38F044D00101795101017219F4
:1048B00008E1010172510101711903E078EC38F04F
:1048C00037D071C100F0016A004A012AE56A800E02
:1048D000E56E0150E56E0050E56EA2EC2CF0006E26
:1048E000040EE12600500101706F010179190CE1FD
:1048F0001F0E01016F1501017A6F7A2B7A2B0101CE
:10490000715101017A277A9F79C100F00101792B59
:10491000016A600E0026000E012200C0E9FF01C0FE
:10492000EAFF6FC1EFFF7951800A02E10101796B63
:10493000E4CF01F0E4CF00F01200D9CFE5FFE1CFE2
:10494000D9FF00C0E5FF01C0E5FF02C0E5FF03C0DD
:10495000E5FF04C0E5FF05C0E5FF06C0E5FF07C0B1
:10496000E5FF08C0E5FF09C0E5FF0AC0E5FF0BC091
:10497000E5FF0CC0E5FF0DC0E5FF0EC0E5FF0FC071
:10498000E5FF020EDBCF00F0030EDBCF01F0040EDB
:10499000DBCF02F0050EDBCF03F0060EDBCF04F019
:1049A000070EDBCF05F0080EDBCF06F0200E076EFA
:1049B000086A06C009F00A6A0B6A0C6AE56AE56AC9
:1049C000E56A0950E56E0350E56E0250E56E015050
:1049D000E56E0050E56EDCEC26F00D6E080EE1266B
:1049E000300E0D263A0E0D5C05E30D500E6E270EAF
:1049F0000E240D6EFF0E07260822D50E07240E6E1C
:104A00000A0E08200F6E0EC0E9FF0FC0EAFF0DC0AE
:104A1000EFFF0C50E56E0B50E56E0A50E56E095045
:104A2000E56E0350E56E0250E56E0150E56E0050F4
:104A3000E56E16EC29F0006EF3CF01F0F4CF02F032
:104A4000E9CF03F0080EE126005001100210031018
:104A5000D8A4AFD707C000F008C001F004C002F02E
:104A600005C003F000C004F001C005F0004A012AAF
:104A7000D50E04260A0E052204C0E9FF05C0EAFF90
:104A8000EFCF04F002C0E9FF03C0EAFF04C0EFFF6C
:104A9000024A032A000E015C02E1200E005CE2E300
:104AA00002C0E9FF03C0EAFF000EEF6AE4CF0FF097
:104AB000E4CF0EF0E4CF0DF0E4CF0CF0E4CF0BF038
:104AC000E4CF0AF0E4CF09F0E4CF08F0E4CF07F038
:104AD000E4CF06F0E4CF05F0E4CF04F0E4CF03F038
:104AE000E4CF02F0E4CF01F0E4CF00F0E4CFD9FF4F
:104AF0001200D9CFE5FFE1CFD9FF00C0E5FF01C02B
:104B0000E5FF02C0E5FF03C0E5FF04C0E5FF05C007
:104B1000E5FF06C0E5FF07C0E5FF08C0E5FF09C0E7
:104B2000E5FF0AC0E5FF0BC0E5FF0CC0E5FF0DC0C7
:104B3000E5FF020EDBCF00F0030EDBCF01F0040E29
:104B4000DBCF02F0050EDBCF03F0060EDBCF04F067
:104B5000070EDBCF05F0080EDBCF06F0090EDBCF2A
:104B600007F0D88003AED890086A083608500FE0E6
:104B7000031C0C6E021C0B6E011C0A6E001C096EDD
:104B8000092A0DE10A2A0BE10B4A0C2A08D000C0C1
:104B900009F001C00AF002C00BF003C00CF0D8808D
:104BA00007AED890006A003600500FE0071C0D6E6B
:104BB000061C036E051C026E041C016E012A0DE129
:104BC000022A0BE1034A0D2A08D004C001F005C0F7
:104BD00002F006C003F007C00DF00D50E56E035063
:104BE000E56E0250E56E0150E56E0C50E56E0B501F
:104BF000E56E0A50E56E0950E56E16EC29F0016E7F
:104C0000F3CF02F0F4CF03F0E9CF04F0080EE12671
:104C10000050081A085016E0041C076E031C066EAC
:104C2000021C056E011C006E002A04E1052A02E147
:104C3000064A072A07C0E9FF06C0F4FF05C0F3FFD4
:104C4000005007D004C0E9FF03C0F4FF02C0F3FF27
:104C50000150E4CF0DF0E4CF0CF0E4CF0BF0E4CF43
:104C60000AF0E4CF09F0E4CF08F0E4CF07F0E4CF96
:104C700006F0E4CF05F0E4CF04F0E4CF03F0E4CF96
:104C800002F0E4CF01F0E4CF00F0E4CFD9FF12004E
:104C9000D9CFE5FFE1CFD9FF00C0E5FF01C0E5FFB7
:104CA00002C0E5FF03C0E5FF04C0E5FF05C0E5FF66
:104CB00006C0E5FF07C0E5FF020EDBCF00F0030EE4
:104CC000DBCF01F0040EDBCF02F000500B0F036EC0
:104CD000000E0120046E000E0220E56AF46AF66AF6
:104CE000F76A03C0E9FF04C0F3FF3AEC38F0005064
:104CF000070F036E000E0120046E000E0220056EE9
:104D00000050030F066E000E0120076E000E0220F9
:104D1000E56AF46AF66AF76A06C0E9FF07C0F3FFBE
:104D20003AEC38F0E56AF46AF66AF76A03C0E9FF1C
:104D300004C0F3FF05503AEC38F00050010F036E49
:104D4000000E0120046E000E0220056E0050020FBE
:104D5000066E000E0120076E000E0220E56A06C0F6
:104D6000E9FF07C0F3FFB7EC38F0E56A03C0E9FFDD
:104D700004C0F3FF0550B7EC38F0E56A00C0E9FF66
:104D800001C0F3FF0250B7EC38F0E4CF07F0E4CFF6
:104D900006F0E4CF05F0E4CF04F0E4CF03F0E4CF75
:104DA00002F0E4CF01F0E4CF00F0E4CFD9FF12002D
:104DB00025642025640A0000D9CFE5FFE1CFD9FFA3
:104DC00000C0E5FF01C0E5FF02C0E5FF03C0E5FF4D
:104DD00004C0E5FF05C0E5FF06C0E5FF07C0E5FF2D
:104DE00008C0E5FF09C0E5FF0AC0E5FF020EDBCF02
:104DF00000F0030EDBCF01F0040EDBCF02F0050E56
:104E0000DBCF03F0060EDBCF04F0070EDBCF05F09F
:104E1000080EDBCF06F0090EDBCF07F0086A096A3F
:104E20000750800BE8440A6E0A501BE10450042628
:104E30000536063607360750035C08E10650025C6B
:104E400005E10550015C02E10450005C06E2D890E7
:104E5000073206320532043204D0092A09C008F0AC
:104E6000DFD70750035C08E10650025C05E10550FE
:104E7000015C02E10450005C08E30450005E055050
:104E8000015A0650025A0750035AD8900732063288
:104E90000532043208C009F008060950E2E103C0F7
:104EA000E9FF02C0F4FF01C0F3FF0050E4CF0AF0B5
:104EB000E4CF09F0E4CF08F0E4CF07F0E4CF06F048
:104EC000E4CF05F0E4CF04F0E4CF03F0E4CF02F048
:104ED000E4CF01F0E4CF00F0E4CFD9FF120000C02E
:104EE000E5FF01C0E5FF03C0E5FF04C0E5FF05C025
:104EF000E5FF06C0E5FF07C0E5FF08C0E5FF09C004
:104F0000E5FF0AC0E5FF0BC0E5FF60C100F061C12D
:104F100001F00101603F01D0612B0050E56E6AECA9
:104F200038F0E652076E046A056A066A60C100F04E
:104F300061C101F00101603F01D0612B0050E56EBD
:104F40006AEC38F0E6520B6A0A6E086A08500412DE
:104F500005120A5006120B50071260C100F061C121
:104F600001F00101603F01D0612B0050E56E6AEC59
:104F700038F0E652036E006A03C001F0E86A03BE2F
:104F8000FF0E086E096E0050041201500512085001
:104F900006120950071260C100F061C101F0010161
:104FA000603F01D0612B0050E56E6AEC38F0E652AC
:104FB000016A0412015005120612071207C0E9FF28
:104FC00006C0F4FF05C0F3FF0450E4CF0BF0E4CFBC
:104FD0000AF0E4CF09F0E4CF08F0E4CF07F0E4CF23
:104FE00006F0E4CF05F0E4CF04F0E4CF03F0E4CF23
:104FF00001F0E4CF00F0120000C0E5FF01C0E5FFC2
:1050000002C0E5FF03C0E5FF04C0E5FF01017251E6
:105010000101711901E15FD072C100F0002A009E08
:10502000600E0024016E026A000E022201C0E9FF38
:1050300002C0EAFFEFCF7CF11F0E01017C1772C1A5
:105040007BF17C5101017B277B2B7B2B7B9F57ECDA
:1050500035F0016E015003E1016A012A01D0016AB5
:1050600057EC35F001017C6F800E7C15026E1F0E2F
:105070007C15036E03C004F003C07CF1045003E10F
:1050800071C172F13BD001501BE0025022E057EC9D
:1050900035F0006E01017C070050420A1AE0005012
:1050A0004E0A03E1A2EC31F014D00050460A03E1AD
:1050B000ACEC38F00ED00050490A0BE1FF0009D0EB
:1050C00072C17DF1025003E0A3EC32F002D068EC33
:1050D00036F07BC172F1010104510101051906E0AE
:1050E0000101735103E1A2EC29F008D08BB006D086
:1050F0000101735103E1ACB278EC38F0E4CF04F075
:10510000E4CF03F0E4CF02F0E4CF01F0E4CF00F00D
:105110001200D9CFE5FFE1CFD9FF00C0E5FF01C004
:10512000E5FF02C0E5FF03C0E5FF04C0E5FF05C0E1
:10513000E5FF06C0E5FF07C0E5FF08C0E5FF0BC0BF
:10514000E5FF0CC0E5FF0DC0E5FF020EDBCF00F070
:10515000030EDBCF01F0040EDBCF02F0050EDBCF38
:1051600003F0060EDBCF04F003C0E5FF04C0F4FF3C
:1051700000C0E9FF01C0F3FF025094EC38F000508A
:10518000020F056E000E0120066E000E0220076E53
:10519000E86A04BEFF0E086E04500C6E0C2608343C
:1051A0000D6ED8900C360D360344E844FC0B0B6EA4
:1051B0000350E844E844030B0C12E56A0BC0F4FF0B
:1051C0000CC0F6FF0DC0F7FF05C0E9FF06C0F3FFF6
:1051D00007503AEC38F0080E0026000E0122022299
:1051E000E56AF46AF66AF76A00C0E9FF01C0F3FFF6
:1051F00002503AEC38F0E4CF0DF0E4CF0CF0E4CFFD
:105200000BF0E4CF08F0E4CF07F0E4CF06F0E4CFF2
:1052100005F0E4CF04F0E4CF03F0E4CF02F0E4CFF4
:1052200001F0E4CF00F0E4CFD9FF1200D9CFE5FFC1
:10523000E1CFD9FF00C0E5FF01C0E5FF02C0E5FFF7
:1052400003C0E5FF04C0E5FF05C0E5FF06C0E5FFBC
:1052500007C0E5FF08C0E5FF09C0E5FF0AC0E5FF9C
:105260000BC0E5FF0CC0E5FF0DC0E5FF020EDBCF74
:1052700000F0030EDBCF01F0040EDBCF02F0050ED1
:10528000DBCF03F0060EDBCF04F0070EDBCF05F01B
:10529000080EDBCF06F0090EDBCF07F0086A096ABB
:1052A0000A6A0B6A200E0C6E0350800BE8440D6EE8
:1052B000005000260136023603360850082609360B
:1052C0000A360B360D50D8A4088007500B5C08E155
:1052D00006500A5C05E10550095C02E10450085CD7
:1052E00009E30450085E0550095A06500A5A07504F
:1052F0000B5A00800C2ED8D703C0E9FF02C0F4FF80
:1053000001C0F3FF0050E4CF0DF0E4CF0CF0E4CF88
:105310000BF0E4CF0AF0E4CF09F0E4CF08F0E4CFDB
:1053200007F0E4CF06F0E4CF05F0E4CF04F0E4CFDB
:1053300003F0E4CF02F0E4CF01F0E4CF00F0E4CFDB
:10534000D9FF120000C0E5FF01C0E5FF02C0E5FF84
:1053500003C0E5FFACA276D0ABEC36F0006E005097
:1053600005E10101056B0101046B6CD005C101F081
:1053700000500126ABEC36F0026E00060250230A04
:105380001FE1010E005CD8A05BD0ABEC36F0026EE2
:10539000690A03E1D2EC34F053D00250720A03E1FF
:1053A00078EC38F04DD00250730A01E049D08B8080
:1053B000AB869D8A9D98AE50AE50AB98AB8840D0DE
:1053C0000250430A05E00250420A01E039D001D000
:1053D000008E00C075F100500F01006F010E010139
:1053E000766F01010551011814E0ABEC36F0026E46
:1053F00001017527000E01017625006E036A0F0E6C
:10540000032200C0E9FF03C0EAFF02C0EFFF762BD2
:10541000E8D7000E01017625006E026A0F0E022207
:105420000101751D036E032A00C0E9FF02C0EAFFF7
:1054300003C0EFFF0101762B76C173F101016D6BA3
:1054400001C005F1E4CF03F0E4CF02F0E4CF01F0B6
:10545000E4CF00F01200D9CFE5FFE1CFD9FF00C0C3
:10546000E5FF01C0E5FF02C0E5FF03C0E5FF04C0A2
:10547000E5FF05C0E5FF06C0E5FF07C0E5FF020E3A
:10548000DBCF00F0030EDBCF01F0040EDBCF02F028
:10549000050EDBCF03F002C006F00650046E800A52
:1054A00033E100C0E9FF01C0F3FF025005EC37F023
:1054B000056EF3CF06F0F4CF07F003C0E5FF05C09B
:1054C000E9FF06C0F3FF0750B7EC38F000C0E9FF72
:1054D00001C0F3FF025005EC37F0056EF3CF06F084
:1054E000F4CF07F0052A02E3064A072A05C0E5FFC4
:1054F00006C0F4FF07C0F6FF00C0E9FF01C0F3FFDC
:1055000002505BEC38F01DD004AA1BD0047A045082
:1055100004E10350F0EC38F014D00450010A04E127
:10552000035002EC00F00DD004500F0A04E10350C8
:10553000A1EC34F006D004500E0A03E1035000EC55
:1055400039F0E4CF07F0E4CF06F0E4CF05F0E4CF84
:1055500004F0E4CF03F0E4CF02F0E4CF01F0E4CFB5
:1055600000F0E4CFD9FF1200D9CFE5FFE1CFD9FF9A
:1055700000C0E5FF01C0E5FF02C0E5FF03C0E5FF95
:1055800004C0E5FF05C0E5FF06C0E5FF07C0E5FF75
:1055900008C0E5FF09C0E5FF0AC0E5FF0BC0E5FF55
:1055A0000CC0E5FF020EDBCF00F0030EDBCF01F0F5
:1055B000040EDBCF02F0050EDBCF03F0060EDBCFCF
:1055C00004F0070EDBCF05F0080EDBCF06F0090E66
:1055D000DBCF07F002500A6E0150096E0050086ED2
:1055E00006C00BF007C00CF0FF0E062607220B507A
:1055F0000C101AE003C0E9FF04C0F3FF055029ECCA
:1056000038F00B6E032A02E3044A052A0BC0E5FFBB
:1056100008C0E9FF09C0F3FF0A50B7EC38F0082AC8
:10562000DFE3094A0A2ADCD702C0F4FF01C0F3FF16
:105630000050E4CF0CF0E4CF0BF0E4CF0AF0E4CF5D
:1056400009F0E4CF08F0E4CF07F0E4CF06F0E4CFB0
:1056500005F0E4CF04F0E4CF03F0E4CF02F0E4CFB0
:1056600001F0E4CF00F0E4CFD9FF1200D9CFE5FF7D
:10567000E1CFD9FF00C0E5FF01C0E5FF02C0E5FFB3
:1056800003C0E5FF04C0E5FF05C0E5FF06C0E5FF78
:1056900007C0E5FF020EDBCF00F0030EDBCF01F009
:1056A000040EDBCF02F0050EDBCF03F005C106F1DF
:1056B000010104510101065F060703C004F0056AF9
:1056C000030E0426D8B0052A06C106F0076A075063
:1056D000800FF36E0550800FF35C02E10450065C0E
:1056E00002E2E8682BD0020E035C02E2E86A26D0F0
:1056F00003060350E56E1DEC33F0E652046A0350D6
:10570000045C14E204500024056EE86A0120066E71
:10571000E86A022005C0E9FF06C0F3FF29EC38F073
:10572000042AE56E1DEC33F0E652E9D705C106F117
:10573000010104510101065F0607E86AE4CF07F0A2
:10574000E4CF06F0E4CF05F0E4CF04F0E4CF03F0BB
:10575000E4CF02F0E4CF01F0E4CF00F0E4CFD9FFD2
:10576000120000C0E5FF01C0E5FF02C0E5FF03C075
:10577000E5FF04C0E5FF006A620E0024016E026AC4
:10578000010E022201C0E9FF02C0EAFFEF6A002A0F
:10579000020E005CF1E3006A016A026AE00E012475
:1057A000036E000E0220046E03C0E9FF04C0EAFF8E
:1057B000EE6AEF6A5C0E0124036E040E0220046E92
:1057C00003C0E9FF04C0EAFFEE6AEF6A550E012448
:1057D000036E0A0E0220046E03C0E9FF04C0EAFF54
:1057E000EE6AEF6A750E0124036E0A0E0220046E43
:1057F00003C0E9FF04C0EAFFEE6AEF6A950E0124D8
:10580000036E0A0E0220046E03C0E9FF04C0EAFF23
:10581000EE687F0EEF6E020E0126D8B0022A002A33
:10582000100E005CD8A0BAD7AF0EC06EC16A010ED0
:10583000C26EC282E4CF04F0E4CF03F0E4CF02F002
:10584000E4CF01F0E4CF00F01200432041202564B2
:105850002025640A0000D9CFE5FFE1CFD9FF00C0C1
:10586000E5FF01C0E5FF02C0E5FF03C0E5FF04C09E
:10587000E5FF05C0E5FF020EDBCF00F0030EDBCF36
:1058800001F0040EDBCF02F00050020DF450036E65
:10589000F3CF00F05C0E0024046E040E0320056EAE
:1058A00004C0E9FF05C0EAFF01C0EEFF02C0EFFF40
:1058B000550E0024046E0A0E0320056E04C0E9FF95
:1058C00005C0EAFFEECF04F0EFCF05F00150045C15
:1058D000016E02500558026EB50E00260A0E032214
:1058E00000C0E9FF03C0EAFF01C0EEFF02C0EFFF06
:1058F000D88002AED89004E3021E016CD8B4022A0C
:105900000250800F800F02E1030E015C02E2016A87
:10591000026A0150021007E100C0E9FF03C0EAFF7C
:10592000000EEE6AEF6AE4CF05F0E4CF04F0E4CFB6
:1059300003F0E4CF02F0E4CF01F0E4CF00F0E4CFD5
:10594000D9FF1200D9CFE5FFE1CFD9FF00C0E5FFB5
:1059500001C0E5FF02C0E5FF03C0E5FF04C0E5FFAD
:1059600005C0E5FF06C0E5FF020EDBCF00F0030E29
:10597000DBCF01F0040EDBCF02F0050EDBCF03F02E
:10598000D88001AED890046A0436045007E0011CA8
:10599000066E001C056E054A062A04D000C005F0FC
:1059A00001C006F0D88003AED89007E3031C016E57
:1059B000021C006E004A012A04D002C000F003C09D
:1059C00001F00150E56E0050E56E0650E56E0550A1
:1059D000E56E0BEC2FF0006EF3CF01F0040EE12624
:1059E00004500AE0011C036E001C026E024A032AE6
:1059F00003C0F3FF025003D001C0F3FF0050E4CF17
:105A000006F0E4CF05F0E4CF04F0E4CF03F0E4CFF8
:105A100002F0E4CF01F0E4CF00F0E4CFD9FF1200B0
:105A2000D9CFE5FFE1CFD9FF00C0E5FF01C0E5FF19
:105A300002C0E5FF03C0E5FF04C0E5FF05C0E5FFC8
:105A4000020EDBCF00F0030EDBCF01F0040EDBCF44
:105A500002F0050EDBCF03F060C104F061C105F078
:105A60000101603F01D0612B0350E56E0450E56EEB
:105A7000A8EC35F0E652E65260C104F061C105F0D1
:105A80000101603F01D0612B0250056EE56E0450AC
:105A9000E56EA8EC35F0E652E65260C104F061C153
:105AA00005F00101603F01D0612B0150056EE56EEC
:105AB0000450E56EA8EC35F0E652E65260C104F001
:105AC00061C105F00101603F01D0612B0050E56E1E
:105AD0000450E56EA8EC35F0E652E652E4CF05F04E
:105AE000E4CF04F0E4CF03F0E4CF02F0E4CF01F020
:105AF000E4CF00F0E4CFD9FF1200D9CFE5FFE1CF2A
:105B0000D9FF00C0E5FF01C0E5FF02C0E5FF03C00B
:105B1000E5FF04C0E5FF05C0E5FF06C0E5FF020E96
:105B2000DBCF00F0030EDBCF01F0040EDBCF02F081
:105B300001016C5119E16FEC27F0036EF3CF04F013
:105B4000F4CF05F0E9CF06F003C0E5FF04C0F4FF91
:105B500005C0F6FF06C0F7FF00C0E9FF01C0F3FF74
:105B600002503AEC38F01ED001016C51010A1AE1E2
:105B700000C0E9FF01C0F3FF02508BEC36F0006E6D
:105B8000F3CF01F0F4CF02F0E9CF03F00350E56E5C
:105B90000250E56E0150E56E0050E56E10EC2DF000
:105BA000040EE126E4CF06F0E4CF05F0E4CF04F0E4
:105BB000E4CF03F0E4CF02F0E4CF01F0E4CF00F053
:105BC000E4CFD9FF1200D9CFE5FFE1CFD9FF00C064
:105BD000E5FF01C0E5FF02C0E5FF03C0E5FF04C02B
:105BE000E5FF020EDBCF00F0030EDBCF01F0040E69
:105BF000DBCF02F00050070F036E000E0120046E91
:105C0000000E0220E56E0450E56E0350E56E64EC74
:105C100032F0030EE1260050230F036E000E012028
:105C2000046E000E0220E56E0450E56E0350E56E32
:105C3000BFEC2FF0030EE1260050330F036E000E71
:105C40000120046E000E0220E56E0450E56E035044
:105C5000E56EACEC2EF0030EE126440E0026000E9D
:105C6000012202220250E56E0150E56E0050E56E01
:105C7000ACEC2EF0030EE126E4CF04F0E4CF03F009
:105C8000E4CF02F0E4CF01F0E4CF00F0E4CFD9FF9D
:105C90001200D9CFE5FFE1CFD9FF00C0E5FF01C079
:105CA000E5FF02C0E5FF03C0E5FF04C0E5FF05C056
:105CB000E5FF06C0E5FF020EDBCF00F0030EDBCFF1
:105CC00001F0040EDBCF02F0050EDBCF03F0060E71
:105CD000DBCF04F0070EDBCF05F0080EDBCF06F0BC
:105CE000D88003AED89015E306500A0A12E104C02A
:105CF000E9FF05C0EAFF2D0EEF6E044A052A031ED8
:105D0000021E011E006C05E1012A03E1022AD8B43B
:105D1000032A0650E56E0550E56E0450E56E03500B
:105D2000E56E0250E56E0150E56E0050E56E9DECAB
:105D300024F0070EE126E4CF06F0E4CF05F0E4CF2F
:105D400004F0E4CF03F0E4CF02F0E4CF01F0E4CFBD
:105D500000F0E4CFD9FF1200D9CFE5FFE1CFD9FFA2
:105D600000C0E5FF01C0E5FF02C0E5FF03C0E5FF9D
:105D700004C0E5FF020EDBCF00F0030EDBCF01F025
:105D8000040EDBCF02F00250E56E0150E56E0050CC
:105D9000E56E64EC32F0030EE1260050010F036E55
:105DA000000E0120046E000E0220E56E0450E56E28
:105DB0000350E56E64EC32F0030EE1260050020F52
:105DC000036E000E0120046E000E0220E56E0450EA
:105DD000E56E0350E56E64EC32F0030EE1260F0E23
:105DE0000026000E012202220250E56E0150E56EEF
:105DF0000050E56EBBEC30F0030EE126E4CF04F07A
:105E0000E4CF03F0E4CF02F0E4CF01F0E4CF00F000
:105E1000E4CFD9FF1200D9CFE5FFE1CFD9FF00C011
:105E2000E5FF01C0E5FF02C0E5FF03C0E5FF04C0D8
:105E3000E5FF05C0E5FF06C0E5FF020EDBCF00F081
:105E4000030EDBCF01F0040EDBCF02F0050EDBCF3B
:105E500003F0046A056A0350800BE844066E06509E
:105E600011E10250022603360350015C02E10250A8
:105E7000005C04E2D8900332023204D0052A05C047
:105E800004F0E9D70350015C02E10250005C04E336
:105E90000250005E0350015AD8900332023204C00F
:105EA00005F004060550EEE101C0F3FF0050E4CF19
:105EB00006F0E4CF05F0E4CF04F0E4CF03F0E4CF44
:105EC00002F0E4CF01F0E4CF00F0E4CFD9FF1200FC
:105ED000D9CFE5FFE1CFD9FF00C0E5FF01C0E5FF65
:105EE00002C0E5FF03C0E5FF04C0E5FF05C0E5FF14
:105EF00006C0E5FF020EDBCF00F0030EDBCF01F0A2
:105F00000038E8441F0B026E036A620E0226010E7F
:105F1000032202C0E9FF03C0EAFFEFCF04F0070E3F
:105F20000014056E010E066E055005E0E86CD89071
:105F30000636010FFDE30650041202C0E9FF03C05C
:105F4000EAFF04C0EFFF026A230E00260F0E0222B2
:105F500000C0E9FF02C0EAFF01C0EFFFE4CF06F096
:105F6000E4CF05F0E4CF04F0E4CF03F0E4CF02F097
:105F7000E4CF01F0E4CF00F0E4CFD9FF1200D9CF95
:105F8000E5FFE1CFD9FF00C0E5FF01C0E5FF02C09A
:105F9000E5FF03C0E5FF04C0E5FF020EDBCF00F024
:105FA000030EDBCF01F0040EDBCF02F00050060F32
:105FB000036E000E0120046E000E0220E56E0450F8
:105FC000E56E0350E56EBBEC30F0030EE1260050A9
:105FD0000C0F036E000E0120046E000E0220E56E11
:105FE0000450E56E0350E56EBBEC30F0030EE12685
:105FF0000E0E0026000E012202220250E56E015014
:10600000E56E0050E56EBBEC30F0030EE126E4CF08
:1060100004F0E4CF03F0E4CF02F0E4CF01F0E4CFEA
:1060200000F0E4CFD9FF120000C0E5FF01C0E5FF9A
:1060300002C0E5FF03C0E5FF72C100F0016A7DC147
:1060400002F0036A0250005E0350015AE56A800EB6
:10605000E56E0150E56E0050E56EA2EC2CF0006E8E
:10606000040EE12600067DC101F0430EA1EC34F0E0
:10607000200EA1EC34F00050800F7F0F20E3600E63
:106080000124026E036A000E032202C0E9FF03C06E
:10609000EAFFEFCF02F0E56A0250E56E000EE56E12
:1060A000710EE56E080EE56E24EC32F0050EE12669
:1060B000012A0150800A01E1016A0006DCD7E4CF21
:1060C00003F0E4CF02F0E4CF01F0E4CF00F01200DF
:1060D000D9CFE5FFE1CFD9FF00C0E5FF01C0E5FF63
:1060E00002C0E5FF03C0E5FF04C0E5FF020EDBCF01
:1060F00000F0030EDBCF01F0040EDBCF02F0E56A07
:10610000F46A00C0E9FF01C0F3FF025094EC38F0DC
:106110000050020F036E000E0120046E000E0220DC
:10612000E56AF46AF66AF76A03C0E9FF04C0F3FFA0
:106130003AEC38F0080E0026000E01220222E56A31
:10614000F46AF66AF76A00C0E9FF01C0F3FF025083
:106150003AEC38F0E4CF04F0E4CF03F0E4CF02F0FF
:10616000E4CF01F0E4CF00F0E4CFD9FF12002564C2
:106170002025640A0000D9CFE5FFE1CFD9FF00C098
:10618000E5FF01C0E5FF02C0E5FF03C0E5FF04C075
:10619000E5FF020EDBCF00F0030EDBCF01F0040EB3
:1061A000DBCF02F001016C5111E13BEC34F0036EE6
:1061B000F3CF04F003C0E5FF04C0F4FF00C0E9FF23
:1061C00001C0F3FF025094EC38F016D001016C517D
:1061D000010A12E100C0E9FF01C0F3FF0250C4EC64
:1061E00037F0006EF3CF01F00150E56E0050E56E20
:1061F000E0EC32F0E652E652E4CF04F0E4CF03F0F4
:10620000E4CF02F0E4CF01F0E4CF00F0E4CFD9FF17
:106210001200C80EF66E710EF76E000EF86E0900D1
:10622000F550056E0900F550066E04E1056702D0D1
:1062300056EF31F00900F550006E0900F550016E7F
:106240000900F550026E09000900F550E96E0900D9
:10625000F550EA6E090009000900F550036E0900C7
:10626000F550046E09000900F6CF07F0F7CF08F0EB
:10627000F8CF09F000C0F6FF01C0F7FF02C0F8FF39
:10628000035002E1045007E00900F550EE6E0306EA
:10629000F8E20406F9D707C0F6FF08C0F7FF09C007
:1062A000F8FF050601E2060615EF31F01200D9CF1E
:1062B000E5FFE1CFD9FF00C0E5FF01C0E5FF02C067
:1062C000E5FF03C0E5FF04C0E5FF05C0E5FF020EE2
:1062D000DBCF00F00050010A24E1016A026A036A80
:1062E000750E0224046E0A0E0320056E04C0E9FF39
:1062F00005C0EAFFEE687F0EEF6E950E0224046E75
:106300000A0E0320056E04C0E9FF05C0EAFFEE6A2D
:10631000EF6A020E0226D8B0032A012A100E015C91
:10632000DFE300C00AF1E4CF05F0E4CF04F0E4CFEE
:1063300003F0E4CF02F0E4CF01F0E4CF00F0E4CFCB
:10634000D9FF120000C0E5FF01C0E5FF02C0E5FF74
:1063500057EC35F0006E57EC35F0016E0050026ED0
:10636000D00E0224006E0A0E005C05E30050026E9F
:10637000F90E0224006E0150026ED00E0224016E4E
:106380000A0E015C05E30150026EF90E0224016E53
:10639000080E005C12E2100E015CD8B00ED000387E
:1063A000F00B0124006E94EC33F0016E015005E116
:1063B0000050E56E3AEC37F0E652E4CF02F0E4CF5D
:1063C00001F0E4CF00F01200D9CFE5FFE1CFD9FF13
:1063D00000C0E5FF01C0E5FF02C0E5FF03C0E5FF27
:1063E00004C0E5FF020EDBCF00F00038E8441F0BCD
:1063F000016E026A620E0126010E022201C0E9FF4F
:1064000002C0EAFFEFCF03F0070E0016010E046E84
:10641000005005E0E86CD8900436010FFDE3041C41
:10642000031601C0E9FF02C0EAFF03C0EFFFE4CF9B
:1064300004F0E4CF03F0E4CF02F0E4CF01F0E4CFC6
:1064400000F0E4CFD9FF1200D9CFE5FFE1CFD9FFAB
:1064500000C0E5FF01C0E5FF02C0E5FF020ED92440
:10646000006E000EDA20016E800E026E030E002612
:10647000000E012202220250E56E0150E56E00502E
:10648000E56E040EDBCFE5FF030EDBCFE5FF020E6A
:10649000DBCFE5FF0A01FF51E56EFE51E56EFD51D0
:1064A000E56E12EC05F0006EF3CF01F0090EE12667
:1064B00001C0F3FF0050E4CF02F0E4CF01F0E4CFDD
:1064C00000F0E4CFD9FF1200D9CFE5FFE1CFD9FF2B
:1064D00000C0E5FF01C0E5FF02C0E5FF03C0E5FF26
:1064E000020EDBCF00F0030EDBCF01F0040EDBCF9A
:1064F00002F001016C510DE198EC37F0036E03C01E
:10650000E5FF00C0E9FF01C0F3FF0250B7EC38F02F
:106510000FD001016C51010A0BE100C0E9FF01C07D
:10652000F3FF025029EC38F0E56E1DEC36F0E65230
:10653000E4CF03F0E4CF02F0E4CF01F0E4CF00F0C9
:10654000E4CFD9FF120000C0E5FF01C0E5FF57EC22
:1065500035F0006E4C0A08E157EC35F0300A02E0E5
:106560008B8229D08B9227D00050450A24E1000E5F
:10657000E56E250EE56E3E0EE56E24EC32F0030E60
:10658000E126FAEC38F0006E00C001F00006015080
:106590000FE057EC35F0E56AE56E000EE56E250E6E
:1065A000E56E400EE56E24EC32F0050EE126ECD7E8
:1065B0000A0EA1EC34F0E4CF01F0E4CF00F01200B9
:1065C000D9CFE5FFE1CFD9FF00C0E5FF01C0E5FF6E
:1065D00002C0E5FF03C0E5FF020EDBCF00F0030EB3
:1065E000DBCF01F060C102F061C103F00101603F47
:1065F00001D0612B0150E56E0250E56EA8EC35F03C
:10660000E652E65260C102F061C103F00101603F51
:1066100001D0612B0050E56E0250E56EA8EC35F01C
:10662000E652E652E4CF03F0E4CF02F0E4CF01F00B
:10663000E4CF00F0E4CFD9FF1200D9CFE5FFE1CFDE
:10664000D9FF00C0E5FF01C0E5FF02C0E5FF03C0C0
:10665000E5FF04C0E5FF020EDBCF00F004C101F04E
:10666000026A014A022A05C103F0046A01500318B4
:1066700003E10250041801E001D00ED0000E010128
:106680000425016E026A070E022201C0E9FF02C062
:10669000EAFF00C0EFFF042BE4CF04F0E4CF03F0E7
:1066A000E4CF02F0E4CF01F0E4CF00F0E4CFD9FF73
:1066B0001200D9CFE5FFE1CFD9FF00C0E5FF01C04F
:1066C000E5FF02C0E5FF03C0E5FF020EDBCF00F0EF
:1066D000016A7DC102F0036A0250002603500122C4
:1066E000E56A800EE56E0150E56E0050E56EA2ECA5
:1066F0002CF0006EF3CF01F0040EE126600E0026B0
:10670000000E012200C0E9FF01C0EAFFEFCF00F058
:106710000050E4CF03F0E4CF02F0E4CF01F0E4CF87
:1067200000F0E4CFD9FF120000C0E5FF01C0E5FF93
:1067300002C0E5FF010E006E57EC35F0016E01C09E
:1067400002F0015023E00050E56E6AEC38F0016E73
:10675000E652015010E10A0E005C0BE20A0E006ED8
:10676000E56E6AEC38F0016EE652015004E1E8682B
:106770000ED0E8680CD00150021802E0E86807D09B
:10678000002A1B0E005CD8E3E86801D0E86AE4CF79
:1067900002F0E4CF01F0E4CF00F01200F3CFE5FF08
:1067A000F4CFE5FFE9CFE5FFEACFE5FFFACFE5FF5C
:1067B000FBCFE5FF010102510F01356F01010351CC
:1067C0000F01366FD650336FD750346FF2A411D00B
:1067D0000101023F01D0032BF294010102510F018C
:1067E000356F010103510F01366FD650336FD7500B
:1067F000346FE4CFFBFFE4CFFAFFE4CFEAFFE4CF4E
:10680000E9FFE4CFF4FFE4CFF3FF1100D9CFE5FFB8
:10681000E1CFD9FF00C0E5FF01C0E5FF02C0E5FF01
:1068200003C0E5FF04C0E5FF020EDBCF00F0030E5E
:10683000DBCF01F0040EDBCF02F0050EDBCF03F05F
:10684000060EDBCF04F003C0E5FF04C0F4FF00C078
:10685000E9FF01C0F3FF025094EC38F0E4CF04F0FC
:10686000E4CF03F0E4CF02F0E4CF01F0E4CF00F096
:10687000E4CFD9FF120000C0E5FF01C0E5FF02C070
:10688000E5FF03C0E5FF60C100F061C101F0010157
:10689000603F01D0612B0050E56E6AEC38F0E652A3
:1068A000036E026A60C100F061C101F00101603F46
:1068B00001D0612B0050E56E6AEC38F0E652016AB7
:1068C00002120150031203C0F3FF0250E4CF03F0A1
:1068D000E4CF02F0E4CF01F0E4CF00F01200D9CF12
:1068E000E5FFE1CFD9FF00C0E5FF01C0E5FF02C031
:1068F000E5FF03C0E5FF04C0E5FF020EDBCF00F0BB
:10690000030EDBCF01F0040EDBCF02F0050EDBCF70
:1069100003F0060EDBCFE9FF070EDBCFEAFF080E20
:10692000DBCF04F0D6EC0CF0E4CF04F0E4CF03F0BE
:10693000E4CF02F0E4CF01F0E4CF00F0E4CFD9FFE0
:10694000120000C0E5FF01C0E5FF02C0E5FF006ED8
:10695000390E01010925016E026A040E022201C0EE
:10696000E9FF02C0EAFF00C0EFFF220E095D01E26D
:10697000092B00500A0A0FE101010951E56E800E52
:10698000E56E040EE56E390EE56E36EC2BF0040E66
:10699000E1260101096BE4CF02F0E4CF01F0E4CF7E
:1069A00000F012000101046B0101056B0101066991
:1069B0008B809490B06A3F0EAF6EB886AC8AAC8480
:1069C000AC8CAC90AB8CAB8E0101746B01016E6B27
:1069D0000101716B0101726B0101736B000EE56ABD
:1069E0006AEC38F00101086FE6529F989F9A010EF9
:1069F0000101076F0A01FD6BFE6B2F0EFF6F78EC34
:106A000038F01200D9CFE5FFE1CFD9FF00C0E5FF94
:106A100001C0E5FF02C0E5FF03C0E5FF020EDBCFCA
:106A200000F0030EDBCF01F0040EDBCF02F0050E09
:106A3000DBCF03F0060EDBCFE9FF070EDBCFEAFF6B
:106A400031EC1BF0E4CF03F0E4CF02F0E4CF01F02F
:106A5000E4CF00F0E4CFD9FF12000101025104019C
:106A60008C6F0101035104018D6FD6508A6FD7508E
:106A70008B6F8C510101021905E104018D51010157
:106A800003190CE00101025104018C6F0101035153
:106A900004018D6FD6508A6FD7508B6F8DC4E9FF7C
:106AA0008CC4F4FF8BC4F3FF04018A51120000C0B0
:106AB000E5FF01C0E5FF0101725101017B1905E00D
:106AC000010172510101711902E1E86A15D072C128
:106AD00000F00101722B016A600E0026000E0122F7
:106AE00000C0E9FF01C0EAFFEFCF00F07251800A59
:106AF00002E10101726B0050E4CF01F0E4CF00F03D
:106B0000120000C0E5FFF4EC38F00401896B806BE3
:106B10008983006A89B3002A0050010BE844F46EAF
:106B20008051FD0BF410806FD58ED59CD59AD588F9
:106B3000D596D594D582D580F28AF184D08EF28E06
:106B4000F28CBA80FF0EBB68BA84E4CF00F012006A
:106B5000D9CFE5FFE1CFD9FF00C0E5FF020EDBCFC3
:106B600000F0030EDBCFA8FF00C0A9FFA69EA69CE5
:106B7000A684F29EF29C550EA76EAA0EA76EA68260
:106B8000A6A202D00000FCD7E86AA6B6E82AA6941E
:106B9000F28EF28CE4CF00F0E4CFD9FF1200D9CF0F
:106BA000E5FFE1CFD9FF00C0E5FF01C0E5FF020E20
:106BB000DBCF00F00050020DF450016EF3CF00F077
:106BC000B50E00260A0E012200C0E9FF01C0EAFF4F
:106BD000EECF00F0EFCF01F001C0F3FF0050E4CFA3
:106BE00001F0E4CF00F0E4CFD9FF1200D9CFE5FFE8
:106BF000E1CFD9FF00C0E5FF01C0E5FF020EDBCF0A
:106C000000F00050020DF450016EF3CF00F0E00EE2
:106C10000026000E012200C0E9FF01C0EAFFEECF0E
:106C200000F0EFCF01F001C0F3FF0050E4CF01F01E
:106C3000E4CF00F0E4CFD9FF1200D9CFE5FFE1CFD8
:106C4000D9FF00C0E5FF01C0E5FF02C0E5FF020E6D
:106C5000DBCF00F060C101F061C102F00101603FD3
:106C600001D0612B0050E56E0150E56EA8EC35F0C7
:106C7000E652E652E4CF02F0E4CF01F0E4CF00F0B8
:106C8000E4CFD9FF1200D8CFE5FFE0CFE5FFE56EF6
:106C9000F3CFE5FFF4CFE5FFE9CFE5FFEACFE5FF6E
:106CA000FACFE5FFFBCFE5FF9BEC23F0E4CFFBFF42
:106CB000E4CFFAFFE4CFEAFFE4CFE9FFE4CFF4FF4B
:106CC000E4CFF3FFE450E4CFE0FFE4CFD8FF1000BF
:106CD00000C0E5FF57EC35F0006E780A04E0005084
:106CE000790A0CE015D0800EE56E040EE56E930E69
:106CF000E56E4AEC19F0030EE1260AD0800EE56E2F
:106D00000A0EE56E000EE56E4AEC19F0030EE12660
:106D1000E4CF00F01200E8AE0AD0F3CFEAFFEE5065
:106D2000EECFF3FFEECFF4FFEECFE9FF1200E8BCA9
:106D30000DEF39F0E9CFF6FFF3CFF7FFF86E09005A
:106D4000F5500900F5CFF3FF0900F5CFF4FF090076
:106D5000F5CFE9FF120000C0E5FF01C0E5FF01012A
:106D600004510101051902E1E86A0FD0000E01018A
:106D70000525006E016A070E012200C0E9FF01C06F
:106D8000EAFFEFCF00F0052B0050E4CF01F0E4CF95
:106D900000F01200F2CFEAFFF29EA69EA69CA68407
:106DA000E9CFA9FFF3CFAAFFE4CFA8FFCCEC38F0DE
:106DB000F4CFA8FFCCEC38F0F6CFA8FFCCEC38F03D
:106DC000F7CFA8FFCCEC38F0A694EABEF28E120002
:106DD000F2CFF6FFF29EA69EA69CE9CFA9FFF3CFC5
:106DE000AAFFA680A850A94AAA2AA680A8CFF3FF86
:106DF000A94AAA2AA680A8CFF4FFA94AAA2AA6804F
:106E0000A8CFEAFFF6BEF28E1200E8AE08D0F3CFAC
:106E1000EAFFEE50EECFF3FFEECFF4FF1200E8BC36
:106E20000FEF39F0E9CFF6FFF3CFF7FFF86E090067
:106E3000F5500900F5CFF3FF0900F5CFF4FF12007C
:106E4000F2CFEAFFF29EA69EA69CA684E9CFA9FFF8
:106E5000F3CFAAFFE4CFA8FFCCEC38F0F4CFA8FF23
:106E6000CCEC38F0F6CFA8FFCCEC38F0A694EABE14
:106E7000F28E1200D9CFE5FFE1CFD9FF00C0E5FFC8
:106E8000020EDBCF00F000C008F10050E56E000EEE
:106E9000E56AA8EC35F0E652E652E4CF00F0E4CF24
:106EA000D9FF1200F2CFF6FFF29EA69EA69CE9CF74
:106EB000A9FFF3CFAAFFA680A850A94AAA2AA680B4
:106EC000A8CFF3FFA94AAA2AA680A8CFF4FFF6BE4E
:106ED000F28E120000C0E5FF01C0E5FF600E010167
:106EE0007225006E016A000E012200C0E9FF01C098
:106EF000EAFFEFCF00F00050E4CF01F0E4CF00F064
:106F00001200D9CFE5FFE1CFD9FF00C0E5FF020EA7
:106F1000DBCF00F0610E005C05E37B0E005C02E25B
:106F2000010E01D0E86AE4CF00F0E4CFD9FF1200EF
:106F300000C0E5FF01C0E5FF60C100F061C101F0E4
:106F40000101603F01D0612B0050E56E6AEC38F022
:106F5000E652E4CF01F0E4CF00F01200D9CFE5FF14
:106F6000E1CFD9FF00C0E5FF020EDBCF00F000C08B
:106F700007F1005004E178EC38F09D9A9D98E4CF39
:106F800000F0E4CFD9FF1200E8AE06D0F3CFEAFF5D
:106F9000EE50EECFF3FF1200E8BC0BEF39F0E9CF73
:106FA000F6FFF3CFF7FFF86E0900F5500900F5CFB3
:106FB000F3FF1200F2CFEAFFF29EA69EA69CA684E3
:106FC000E9CFA9FFF3CFAAFFE4CFA8FFCCEC38F0BC
:106FD000F4CFA8FFCCEC38F0A694EABEF28E1200F3
:106FE00018EEFFF028EEFFF0F86AA68EA69CE9687E
:106FF0000E0EEA6E0068000EED6A0050FDE109EC2D
:1070000031F006EC00F0FFD7F2CFF6FFF29EA69E1D
:10701000A69CE9CFA9FFF3CFAAFFA680A850A94A52
:10702000AA2AA680A8CFF3FFF6BEF28E1200F2CFF6
:10703000EAFFF29EA69EA69CA684E9CFA9FFF3CF05
:10704000AAFFE4CFA8FFCCEC38F0A694EABEF28EFB
:107050001200E8AE04D0F3CFEAFFEE501200E8BC15
:1070600009EF39F0E9CFF6FFF3CFF7FFF86E09002B
:10707000F5501200E8AE0BD0F3CFEAFFE4CFEEFFFD
:10708000F4CFEEFFF6CFEEFFF7CFEEFF1200E8BC35
:1070900007EF39F01200000000000000FF000000C0
:1070A0000007000200000042000000000000000095
:1070B000000000000000E8AE09D0F3CFEAFFE4CF03
:1070C000EEFFF4CFEEFFF6CFEEFF1200E8BC11EFBB
:1070D00039F01200D9CFE5FFE1CFD9FF020EDBCFA7
:1070E000A9FFA69CA69EA680A850E4CFD9FF1200B7
:1070F000ACA2FED78B80AE500000AE50AB98AB88F0
:10710000AB869D8A9D98120025642000F2CFF6FF81
:10711000F29EA69EA69CE9CFA9FFF3CFAAFFA68068
:10712000A850F6BEF28E1200E8AE07D0F3CFEAFF09
:10713000E4CFEEFFF4CFEEFF1200E8BC05EF39F02C
:107140001200700ED36E9B8CFF0E92689368946849
:107150009668626AF19E120000C0E5FF94EC33F07D
:10716000006E005001E1FF00E4CF00F01200E8AE35
:1071700005D0F3CFEAFFE4CFEEFF1200E8BC03EF47
:1071800039F01200D9CFE5FFE1CFD9FF020EDBCFF6
:107190000DF1E4CFD9FF1200550EA76EAA0EA76E0F
:1071A000A682A6B2FED7A94AAA2A010E01016C6FD7
:1071B0001C0E0101606F616B120001016C6B1C0EF3
:1071C0000101606F616B1200010096700000000108
:1071D00000001F00000081EC35F0D2EC34F012000A
:1071E000ACA2FED7AD6E1200A1EC38F01200010186
:1071F0007251120001017C5112000101075112006D
:10720000E8CF7FFF120017EF38F0DAEF37F0CAEF60
:1072100036F086EF38F004EF38F0E8EF36F052EF52
:0672200037F020EF37F00B
:00000001FF
